:100000000C942A001895000018950000189500001F
:10001000189500001895000018950000189500002C
:10002000189500001895000018950000189500001C
:10003000189500001895000018950000189500000C
:1000400018950000189500001895000018950000FC
:10005000189500008FE58DBFC0EEE8EF4E2E88E0CA
:100060008EBFD7E0F6E05F2EEEEFF7E0A0E6B0E05F
:1000700088278D933197E9F766248FE38ABB0E9426
:10008000303186E086B980E487B9D09AD19AD29A85
:10009000D39AD49AD59AD798B898B998BA98BC9A5E
:1000A0008B9A8C9A8D9A8E9AC09AC19AC29A969877
:1000B000C4980108080000000000000000000000D3
:1000C000065F06000000000703000703000000248D
:1000D0007E247E24000000242B6A120000000063AE
:1000E00013086463000000364956205000000000E9
:1000F00007030000000000003E4100000000000077
:10010000413E0000000000083E1C3E0800000008C0
:10011000083E080800000000E06000000000000841
:1001200008080808000000006060000000000020CF
:10013000100804020000003E5149453E0000000046
:10014000427F400000000062514949460000002201
:10015000494949360000001814127F100000002F92
:10016000494949310000003C4A494930000000013A
:1001700071090503000000364949493600000006B0
:100180004949291E000000006C6C000000000000BE
:10019000EC6C000000000008142241000000002464
:1001A000242424240000000041221408000000023E
:1001B000015909060000003E415D551E0000007E09
:1001C0001111117E0000007F494949360000003EB0
:1001D000414141220000007F4141413E0000007F3B
:1001E000494949410000007F090909010000003E1A
:1001F0004149497A0000007F0808087F000000009C
:10020000417F4100000000304040403F0000007F3F
:10021000081422410000007F404040400000007F61
:100220000204027F0000007F0204087F0000003EFD
:100230004141413E0000007F090909060000003EDF
:100240004151215E0000007F090919660000002667
:100250004949493200000001017F01010000003FCF
:100260004040403F0000001F2040201F0000003F92
:10027000403C403F00000063140814630000000786
:1002800008700807000000714945430000000000A5
:100290007F4141000000000204081020000000001F
:1002A00041417F0000000004020102040000808040
:1002B0008080808080800000030700000000002014
:1002C000545454780000007F4444443800000038FF
:1002D00044444428000000384444447F000000386F
:1002E00054545408000000087E090900000000185A
:1002F000A4A4A47C0000007F040478000000000097
:10030000007D40000000004080847D000000007FF0
:100310001028440000000000007F40000000007C26
:10032000041804780000007C040478000000003801
:1003300044444438000000FC444444380000003881
:10034000444444FC000000447844040800000008D1
:1003500054545420000000043E4424000000003C9B
:1003600040207C000000001C2040201C0000003CBD
:100370006030603C0000006C10106C000000009CBD
:10038000A0603C000000006454544C0000000008D1
:100390003E41410000000000007700000000000026
:1003A00041413E0800000002010201000000003C43
:1003B0002623263C0000001EA1E121120000003D82
:1003C00040207D00000000385454550900000020F2
:1003D00055555578000000205554557800000020F0
:1003E0005555547800000020575557780000001CE0
:1003F000A2E22214000000385555550800000038CC
:1004000055545508000000385555540800000000A8
:10041000017C410000000000027942000000000061
:10042000017C400000000070292429700000007841
:100430002F252F780000007C5454554500000034CF
:10044000547C54580000007E097F49490000003860
:1004500045453900000000384544390000000039A6
:10046000454438000000003C41217D000000003D73
:1004700041207C000000009CA1603D000000003D88
:1004800042423D000000003C41403D000000001899
:1004900024662400000000483E494962000000290B
:1004A0002A7C2A290000007F0916781000000040ED
:1004B000887E090200000020545555780000000095
:1004C000007D410000000038444539000000003C38
:1004D00040217D000000007A090A71000000007AC6
:1004E00011227900000000085555555E0000004EAD
:1004F00051514E0000000030484D40200000003CAB
:1005000004040404000004040404041C0000001794
:10051000084C6A500000001708342A7800000000D8
:10052000307D3000000000081400081400000014A2
:100530000800140800004411441144110000AA5599
:10054000AA55AA550000BBEEBBEEBBEE00000000B2
:1005500000FF00000000080808FF000000000A0A71
:100560000AFF0000000008FF00FF0000000008F87C
:1005700008F8000000000A0A0AFE000000000AFB5A
:1005800000FF0000000000FF00FF000000000AFA6A
:1005900002FE000000000A0B080F00000000080F18
:1005A000080F000000000A0A0A0F000000000808F7
:1005B00008F8000000000000000F0808000008080C
:1005C000080F08080000080808F8080800000000E4
:1005D00000FF0808000008080808080800000808CC
:1005E00008FF08080000000000FF0A0A000000FFE2
:1005F00000FF08080000000F080B0A0A000000FEB8
:1006000002FA0A0A00000A0B080B0A0A00000AFA9A
:1006100002FA0A0A000000FF00FB0A0A00000A0AA8
:100620000A0A0A0A00000AFB00FB0A0A00000A0A7A
:100630000A0B0A0A0000080F080F080800000A0A3F
:100640000AFA0A0A000008F808F808080000000F73
:10065000080F080800000000000F0A0A0000000050
:1006600000FE0A0A000000F808F80808000008FF69
:1006700000FF080800000A0A0AFB0A0A000008082E
:10068000080F00000000000000F808080000FFFF4D
:10069000FFFFFFFF0000F0F0F0F0F0F00000FFFFC0
:1006A000FF0000000000000000FFFFFF00000F0F30
:1006B0000F0F0F0F0000001824241824000000FE64
:1006C0004A4A34000000007F0101030000000002DC
:1006D0007E027E020000006355496300000000189E
:1006E00024241C04000000FC20201C000000000842
:1006F0000478040000000008557755080000003E0B
:1007000049493E000000004C7202724C0000002279
:100710005559300000000018241824180000001853
:10072000247E24180000001C2A2A2A000000003C15
:1007300002023C000000002A2A2A2A0000000000D1
:10074000242E2400000000514A4A440000000044C6
:100750004A4A51000000000000FC02040000002092
:10076000403F000000000008082A0808000000249C
:100770001224120000000006090906000000000013
:100780001818000000000000080000000000003001
:10079000403E0202000000010E010E0000000009B0
:1007A0000D0A00000000003C3C3C3C00000082EBD5
:1007B00090E0A0E6B0E08D939C9380E092E2A4E705
:1007C000B0E08D939C935A924A92A4E7B0E08D9149
:1007D0009C91A42DB52D8D939C9382E00E94772F40
:1007E0000E94CB21229682E00E94732FA6E0B1E006
:1007F000EEE8F0E70E94A032ACE0B1E0E4E9F0E717
:100800000E94A032A2E1B1E0EAE9F0E70E94A03242
:10081000A8E1B1E0E0EAF0E70E94A032AEE1B1E089
:10082000E6EAF0E70E94A032A4E2B1E0ECEAF0E7E9
:100830000E94A032A6E0B4E0E2E2F0E70E94623556
:10084000AAE0B4E0E6E2F0E70E946235AEE0B4E090
:10085000EAE2F0E70E946235A2E1B4E0EEE2F0E7FE
:100860000E946235A6E1B4E0E2E3F0E70E9462355F
:1008700082E08093260483E080932B01AAE7B0E016
:10088000E6E3F0E70E946235EAE7F0E00E94CB324F
:10089000A2E9B0E0EDE0FF270E944C3685E08093AE
:1008A00096004091960001E0041718F011F00C94A6
:1008B0008704A6E9B0E0AD90BB24AEE7B0E0AA0C97
:1008C000BB1CAA0CBB1CAA0DBB1D0D911D912D912B
:1008D0003C914AE050E060E070E00E94E12FA6E920
:1008E000B0E0AD90BB24AAE7B0E0AA0CBB1CAA0CF8
:1008F000BB1CAA0DBB1D4D935D936D937D938091A1
:10090000960081508093960010F00C945104A7E952
:10091000B0E0EEE8F0E70E94A032ADE9B0E0E4E933
:10092000F0E70E94A032A3EAB0E0EAE9F0E70E9413
:10093000A032A9EAB0E0E0EAF0E70E94A032AFEA14
:10094000B0E0E6EAF0E70E94A032A5EBB0E0ECEA06
:10095000F0E70E94A03281E08093BB0002E310E048
:1009600020E030E0A2E9B0E04D915D916D917C9185
:100970000E948332ACEBB0E00D931D932D933D9319
:10098000A2E8B0E00D911D912D913C91A0ECB0E05A
:100990000D931D932D933C938091E8008068809384
:1009A000E80082E08093E900A2E9B0E00D911D919A
:1009B0002D913C91ACE6B0E00D931D932D933C93AB
:1009C0000E94963182E08093620081E08093630010
:1009D000882780936400E2EBF0E70E94CF2F83E04A
:1009E0008093620081E08093630088278093640095
:1009F000E4ECF0E70E94CF2F84E08093620081E076
:100A000080936300882780936400E6EDF0E70E94FE
:100A1000CF2F85E08093620081E080936300882778
:100A200080936400E8EEF0E70E94CF2F86E0809389
:100A3000620081E080936300882780936400EAEF7E
:100A4000F0E70E94CF2F87E08093620081E08093DF
:100A50006300882780936400ECE0F1E70E94CF2FC9
:100A6000E2E0F0E00E94D62F0E94963106B347E004
:100A70000423A5E6B0E00C9300916500053011F069
:100A80000C949205A2E9B0E00D911D912D913C913D
:100A9000A4ECB0E00D931D932D933C93A2E9B0E03C
:100AA0000D911D912D913C91A8ECB0E00D931D93FB
:100AB0002D933C930EE110E020E030E0A2E9B0E09D
:100AC0004D915D916D917C910E948332ACECB0E0D0
:100AD0000D931D932D933D93A6E8B0E00D911D91CC
:100AE0002D913C91A0EDB0E00D931D932D933C937F
:100AF000A4EDB0E0EAE3F0E70E946235A8EDB0E0D3
:100B0000EAE3F0E70E946235AAE1B4E0EAE2F0E746
:100B10000E946235AEE1B4E0EEE2F0E70E94623599
:100B20000C94CA05E0E0F0E0A4ECB0E094E00E9490
:100B30006C36E4E0F0E0A8ECB0E094E00E946C36A3
:100B4000E8E0F0E0ACECB0E094E00E946C36ECE061
:100B5000F0E0A0EDB0E094E00E946C36E0E1F0E05F
:100B6000A4EDB0E094E00E946C36E4E1F0E0A8ED82
:100B7000B0E094E00E946C36AAE1B4E0E4E2F0E078
:100B800094E00E946C36AEE1B4E0E8E2F0E094E07C
:100B90000E946C3600916500053011F00C94E5055B
:100BA00085E08093620081E08093630088278093D2
:100BB0006400EEE1F1E70E94CF2F06B347E0042383
:100BC000A5E6B0E00C930C94CA050E9496318AEF1A
:100BD00090E00E943E30379AECE2F0E0A0E4B4E00E
:100BE0000E946B368BE080932A0181E080934F0155
:100BF000EAE2F1E0FA93EA930E942923229606B3EF
:100C000047E00423A5E6B0E00C93009165000430B2
:100C100011F00C9428060E946E2FAAE2B1E08C918C
:100C20008F5F8C9300912A01053110F40C941B0600
:100C300085E180932A010E949631EAE2F1E0FA937D
:100C4000EA930E94292322968AEF90E00E943E3088
:100C500000916500063011F00C944C060E946E2F36
:100C600080912A01815080932A0100912A010B3042
:100C700018F011F00C943F068BE080932A010E943B
:100C80009631EAE2F1E0FA93EA930E942923229650
:100C90008AEF90E00E943E3000916500013011F033
:100CA0000C9466060E946E2FEAE2F1E0FA93EA9352
:100CB0000E9438292296EAE2F1E0FA93EA930E9430
:100CC000292322968AEF90E00E943E300091650031
:100CD000033011F00C9480060E946E2FEAE2F1E0DE
:100CE000FA93EA930E94632B2296EAE2F1E0FA93E8
:100CF000EA930E94292322968AEF90E00E943E30D8
:100D000000912A01053111F00C94DF0606B347E08B
:100D10000423A5E6B0E00C9300916500053011F0C6
:100D20000C9494060C9496060C948606E0E0F0E091
:100D3000A4ECB0E094E07BE70E945B36E4E0F0E0F6
:100D4000A8ECB0E094E07BE70E945B36E8E0F0E0DE
:100D5000ACECB0E094E07BE70E945B36ECE0F0E0C6
:100D6000A0EDB0E094E07BE70E945B36E0E1F0E0CC
:100D7000A4EDB0E094E07BE70E945B36E4E1F0E0B4
:100D8000A8EDB0E094E07BE70E945B36E4E2F0E09F
:100D9000AAE1B4E094E07BE70E945B36E8E2F0E091
:100DA000AEE1B4E094E07BE70E945B368BE0809399
:100DB0002A018AEF90E00E943E300C94F2050091E7
:100DC0002A010B3011F00C941A2106B347E00423DA
:100DD000A5E6B0E00C9300916500053011F00C948D
:100DE0001A210E946E2F8AEF90E00E943E300E94EE
:100DF000963181E08093620081E08093630081E01E
:100E000080936400E2E2F1E70E94CF2F82E08093BA
:100E1000620081E080936300882780936400E2E3AE
:100E2000F1E70E94CF2F83E08093620081E08093FE
:100E30006300882780936400EEE3F1E70E94CF2FE0
:100E400084E08093620081E0809363008827809330
:100E50006400EAE4F1E70E94CF2F85E0809362000E
:100E600081E080936300882780936400E6E5F1E7E2
:100E70000E94CF2F86E08093620081E08093630020
:100E8000882780936400EEE5F1E70E94CF2F87E08A
:100E90008093620081E080936300882780936400E0
:100EA000EAE6F1E70E94CF2F88E08093620081E0BC
:100EB00080936300882780936400EAE7F1E70E944B
:100EC000CF2F06B347E00423A5E6B0E00C930091D2
:100ED0006500063011F00C9482070E946E2F8091FD
:100EE0004F01815080934F018091E800806480938E
:100EF000E80000914F01013010F00C94820788E067
:100F000080934F0100916500043011F00C94A0070C
:100F10000E946E2FAFE4B1E08C918F5F8C93809133
:100F2000E80080648093E80000914F01083018F0D9
:100F300011F00C949D070C94A00781E080934F0161
:100F4000A8EEB0E08C9186FB16F00C94220B0E9468
:100F5000963100914F01013011F00C94190881E095
:100F60008093620081E08093630081E0809364005D
:100F7000E2E2F1E70E94CF2F82E08093620081E0FD
:100F800080936300882780936400E2E3F1E70E9486
:100F9000CF2F83E08093620081E0809363008827F5
:100FA00080936400EEE3F1E70E94CF2F84E080930A
:100FB000620081E080936300882780936400EAE404
:100FC000F1E70E94CF2F85E08093620081E080935B
:100FD0006300882780936400E6E5F1E70E94CF2F45
:100FE00086E08093620081E080936300882780938D
:100FF0006400EEE5F1E70E94CF2F87E08093620066
:1010000081E080936300882780936400EAE6F1E73B
:101010000E94CF2F88E08093620081E0809363007C
:10102000882780936400EAE7F1E70E94CF2F0C94B1
:10103000190B023011F00C94870881E08093620054
:1010400081E080936300882780936400E2E2F1E707
:101050000E94CF2F82E08093620081E08093630042
:1010600081E080936400E2E3F1E70E94CF2F83E008
:101070008093620081E080936300882780936400FE
:10108000EEE3F1E70E94CF2F84E08093620081E0DD
:1010900080936300882780936400EAE4F1E70E946C
:1010A000CF2F85E08093620081E0809363008827E2
:1010B00080936400E6E5F1E70E94CF2F86E08093FD
:1010C000620081E080936300882780936400EEE5EE
:1010D000F1E70E94CF2F87E08093620081E0809348
:1010E0006300882780936400EAE6F1E70E94CF2F2F
:1010F00088E08093620081E080936300882780937A
:101100006400EAE7F1E70E94CF2F0C94190B03303B
:1011100011F00C94F50881E08093620081E08093E7
:101120006300882780936400E2E2F1E70E94CF2FFA
:1011300082E08093620081E080936300882780933F
:101140006400E2E3F1E70E94CF2F83E08093620026
:1011500081E08093630081E080936400EEE3F1E737
:101160000E94CF2F84E08093620081E0809363002F
:10117000882780936400EAE4F1E70E94CF2F85E09E
:101180008093620081E080936300882780936400ED
:10119000E6E5F1E70E94CF2F86E08093620081E0D0
:1011A00080936300882780936400EEE5F1E70E9456
:1011B000CF2F87E08093620081E0809363008827CF
:1011C00080936400EAE6F1E70E94CF2F88E08093E5
:1011D000620081E080936300882780936400EAE7DF
:1011E000F1E70E94CF2F0C94190B043011F00C94EE
:1011F000630981E08093620081E080936300882727
:1012000080936400E2E2F1E70E94CF2F82E08093B6
:10121000620081E080936300882780936400E2E3AA
:10122000F1E70E94CF2F83E08093620081E08093FA
:101230006300882780936400EEE3F1E70E94CF2FDC
:1012400084E08093620081E08093630081E080937A
:101250006400EAE4F1E70E94CF2F85E0809362000A
:1012600081E080936300882780936400E6E5F1E7DE
:101270000E94CF2F86E08093620081E0809363001C
:10128000882780936400EEE5F1E70E94CF2F87E086
:101290008093620081E080936300882780936400DC
:1012A000EAE6F1E70E94CF2F88E08093620081E0B8
:1012B00080936300882780936400EAE7F1E70E9447
:1012C000CF2F0C94190B053011F00C94D10981E04B
:1012D0008093620081E0809363008827809364009C
:1012E000E2E2F1E70E94CF2F82E08093620081E08A
:1012F00080936300882780936400E2E3F1E70E9413
:10130000CF2F83E08093620081E080936300882781
:1013100080936400EEE3F1E70E94CF2F84E0809396
:10132000620081E080936300882780936400EAE490
:10133000F1E70E94CF2F85E08093620081E08093E7
:10134000630081E080936400E6E5F1E70E94CF2F1F
:1013500086E08093620081E0809363008827809319
:101360006400EEE5F1E70E94CF2F87E080936200F2
:1013700081E080936300882780936400EAE6F1E7C8
:101380000E94CF2F88E08093620081E08093630009
:10139000882780936400EAE7F1E70E94CF2F0C943E
:1013A000190B063011F00C943F0A81E08093620023
:1013B00081E080936300882780936400E2E2F1E794
:1013C0000E94CF2F82E08093620081E080936300CF
:1013D000882780936400E2E3F1E70E94CF2F83E047
:1013E0008093620081E0809363008827809364008B
:1013F000EEE3F1E70E94CF2F84E08093620081E06A
:1014000080936300882780936400EAE4F1E70E94F8
:10141000CF2F85E08093620081E08093630088276E
:1014200080936400E6E5F1E70E94CF2F86E0809389
:10143000620081E08093630081E080936400EEE5C8
:10144000F1E70E94CF2F87E08093620081E08093D4
:101450006300882780936400EAE6F1E70E94CF2FBB
:1014600088E08093620081E0809363008827809306
:101470006400EAE7F1E70E94CF2F0C94190B0730C4
:1014800011F00C94AD0A81E08093620081E08093BA
:101490006300882780936400E2E2F1E70E94CF2F87
:1014A00082E08093620081E08093630088278093CC
:1014B0006400E2E3F1E70E94CF2F83E080936200B3
:1014C00081E080936300882780936400EEE3F1E776
:1014D0000E94CF2F84E08093620081E080936300BC
:1014E000882780936400EAE4F1E70E94CF2F85E02B
:1014F0008093620081E0809363008827809364007A
:10150000E6E5F1E70E94CF2F86E08093620081E05C
:1015100080936300882780936400EEE5F1E70E94E2
:10152000CF2F87E08093620081E08093630081E0A9
:1015300080936400EAE6F1E70E94CF2F88E0809371
:10154000620081E080936300882780936400EAE76B
:10155000F1E70E94CF2F0C94190B083011F00C9476
:10156000190B81E08093620081E0809363008827FB
:1015700080936400E2E2F1E70E94CF2F82E0809343
:10158000620081E080936300882780936400E2E337
:10159000F1E70E94CF2F83E08093620081E0809387
:1015A0006300882780936400EEE3F1E70E94CF2F69
:1015B00084E08093620081E08093630088278093B9
:1015C0006400EAE4F1E70E94CF2F85E08093620097
:1015D00081E080936300882780936400E6E5F1E76B
:1015E0000E94CF2F86E08093620081E080936300A9
:1015F000882780936400EEE5F1E70E94CF2F87E013
:101600008093620081E08093630088278093640068
:10161000EAE6F1E70E94CF2F88E08093620081E044
:101620008093630081E080936400EAE7F1E70E9421
:10163000CF2F8AEF90E00E943E308091E8008F7BB0
:101640008093E80000916500053011F00C94300B98
:101650000E946E2F8AEF90E00E943E300C94320B75
:101660000C9461078AEF90E00E943E3000914F0198
:10167000053011F00C943E0B0C94DE1400914F01D8
:10168000083011F00C94460B0C94F2050E94963130
:1016900000914F01043011F00C94500B0C94DE14A7
:1016A00000914F01023018F011F00C94590B0C947A
:1016B000DE1400914F01023011F00C94880B81E090
:1016C0008093620081E080936300882780936400A8
:1016D000E2E8F1E70E94CF2F83E08093620081E08F
:1016E00080936300882780936400E4E9F1E70E9417
:1016F000CF2F85E08093620081E08093630088278C
:1017000080936400E6EAF1E70E94CF2F0C945D120B
:10171000033011F00C94C41181E08093620081E0E9
:1017200080936300882780936400E8EBF1E70E94D0
:10173000CF2F82E08093620081E08093630088274E
:1017400080936400E4ECF1E70E94CF2F8091E800E1
:1017500080618093E80087E08093620081E080935D
:10176000630081E080936400E6EDF1E70E94CF2FF3
:1017700088E08093620081E08093630088278093F3
:101780006400E8EEF1E70E94CF2F06B347E00423A0
:10179000A5E6B0E00C9300916500053011F00C94C3
:1017A000D30B0C943B0C00916500043081E008F4ED
:1017B00080E08F9300916500063081E010F009F021
:1017C00080E09F918923882311F40C94390CA8EEB2
:1017D000B0E08C9184FB882780F9809580FBA8EE8F
:1017E000B0E08C9184F98C93A8EEB0E08C9184FBEE
:1017F00016F00C941B0C87E08093620081E08093CC
:10180000630081E080936400E6EDF1E70E94CF2F52
:1018100088E08093620081E0809363008827809352
:101820006400E8EEF1E70E94CF2F8AEF90E00E947B
:101830003E300C94390C87E08093620081E0809305
:101840006300882780936400E6EDF1E70E94CF2FC4
:1018500088E08093620081E08093630081E0809360
:101860006400E8EEF1E70E94CF2F8AEF90E00E943B
:101870003E300C94C50B8AEF90E00E943E30A8EEFB
:10188000B0E08C9184FB16F40C94C00D969A8AEF0C
:1018900090E00E943E300E94963181E08093620089
:1018A00081E080936300882780936400EAEFF1E78A
:1018B0000E94CF2F82E08093620081E080936300DA
:1018C000882780936400ECE0F2E70E94CF2F83E04A
:1018D0008093620081E08093630088278093640096
:1018E000E6EAF1E70E94CF2F06B347E00423A5E61E
:1018F000B0E00C9300916500053011F00C94820C5F
:101900000C94840C0C94740C87E4806487B90E9456
:10191000A632ABE3B4E08D939C93EEE2F0E0ABE350
:10192000B4E07BE70E945A36ECE2F0E0A0E4B4E0D9
:101930000E946B368AEF90E00E943E30E2E9F0E0D0
:101940000E9409330E942D330E946333EEE3F0E7D7
:101950000E9466340E94D433FF27EDE0AEEFB0E082
:101960000E944C3696980E949E228AEF90E00E9438
:101970003E300E94963181E08093620081E0809346
:101980006300882780936400EEE1F2E70E94CF2F86
:1019900082E08093620081E08093630088278093D7
:1019A0006400E0E3F2E70E94CF2F83E080936200BF
:1019B00081E080936300882780936400E2E4F2E78B
:1019C0000E94CF2F84E08093620081E080936300C7
:1019D000882780936400E4E5F2E70E94CF2F85E03A
:1019E0008093620081E08093630088278093640085
:1019F000E6E6F2E70E94CF2F88E08093620081E064
:101A000080936300882780936400E8E7F2E70E94F0
:101A1000CF2FA0EEB6E0E0E4F4E00E94EE350E94A5
:101A2000C72F06B347E00423A5E6B0E00C9300916E
:101A30006500033011F00C94590DA0E4B4E00E944D
:101A4000812FA0E4B4E00D911C91013050E0150706
:101A500010F00C94310D81E090E0A0E4B4E08D939F
:101A60009C9388E08093620081E0809363008827E4
:101A700080936400E4E8F2E70E94CF2F88E080932F
:101A8000620081E080936300882780936400E8E728
:101A9000F2E70E94CF2FA0EEB6E0E0E4F4E00E946F
:101AA000EE350E94C72F86E990E00E943E300C94EC
:101AB0009A0D013011F00C949A0DA0E4B4E00E944C
:101AC0007B2FA0E4B4E00D911C91043F51E0150779
:101AD00018F011F00C946E0D0C94740D84EF91E0DD
:101AE000A0E4B4E08D939C9388E08093620081E051
:101AF00080936300882780936400E4E8F2E70E9403
:101B0000CF2F88E08093620081E080936300882774
:101B100080936400E8E7F2E70E94CF2FA0EEB6E0E2
:101B2000E0E4F4E00E94EE350E94C72F86E990E0E1
:101B30000E943E3000916500053011F00C94BE0DFE
:101B4000ECE2F0E0A0E4B4E07BE70E945A3696981D
:101B500087E4806487B90E94A632ABE2B4E08D933B
:101B60009C93E0E3F0E0ABE2B4E07BE70E945A36FE
:101B70008AEF90E00E943E300C94C00D0C94110D41
:101B8000E2E9F0E00E9409330E942D330E946333A2
:101B9000EEE3F0E70E9466340E94D433FF27EDE0C5
:101BA000AEEFB0E00E944C3696980E949E228AEFDB
:101BB00090E00E943E300E949631EEE2F0E0ABE30E
:101BC000B4E00E946B36ECE2F0E0A0E4B4E00E94E6
:101BD0006B36E0E3F0E0ABE2B4E00E946B36EBE2A0
:101BE000F4E0D190E080FF2400270E942D330E9472
:101BF0006333E2E4F0E70E9466340E94D433FF27A7
:101C0000EDE0AEEFB3E00E944C36EBE2F4E0D190B1
:101C1000E080FF2400270E942D330E9463332F931E
:101C20003F934F935F93EBE3F4E0D190E080FF2488
:101C300000270E942D335F914F913F912F910E9479
:101C40000534FF27EDE0A2E0B4E00E944C36E2E468
:101C5000F0E70E946F34E2E0F4E00E9409330E9452
:101C6000D433FF27EDE0A2E0B4E00E944C36EAE274
:101C7000F0E70E946F34E2E0F4E00E9409330E9432
:101C80007E33FF27EDE0A2E0B4E00E944C36A8E6E8
:101C9000B0E0EAE2F0E70E946235E8E6F0E0A2E0B8
:101CA000B4E00E94E337FF27EDE0A2E0B4E00E9439
:101CB0004C36E0E4F4E0D190E080FF2400270E945D
:101CC0002D330E946333E2E0F4E00E9409330E9466
:101CD000D433FF27EDE0A2E0B4E00E944C36E2E30B
:101CE000F0E70E946F34E2E0F4E00E9409330E94C2
:101CF000D433FF27EDE0A2E0B4E00E944C36A0EE22
:101D0000B6E0AF93BF93E2E0F4E00E9409330E9493
:101D10004D3011E001E0BF91AF910E948935E0EEB6
:101D2000F6E0ABE3B1E00E94473687E080936200C3
:101D300081E080936300882780936400E6E9F2E7FE
:101D40000E94CF2FABE3B1E00E94C92FE2EAF2E795
:101D50000E94CF2FEBE2F4E0D190E080FF24002737
:101D60000E942D330E946333E6E4F0E70E9466345C
:101D70000E940534FF27EDE0A2E0B4E00E944C365B
:101D8000E2E4F0E70E946F34E2E0F4E00E940933FD
:101D90000E94D433FF27EDE0A2E0B4E00E944C366D
:101DA000EAE2F0E70E946F34E2E0F4E00E940933D7
:101DB0000E947E33FF27EDE0A2E0B4E00E944C36A3
:101DC000E8E6F0E0A2E0B4E00E94E337FF27EDE0B0
:101DD000A2E0B4E00E944C36E0E4F4E0D190E08070
:101DE000FF2400270E942D330E946333E2E0F4E0D9
:101DF0000E9409330E94D433FF27EDE0A2E0B4E053
:101E00000E944C36E2E3F0E70E946F34E2E0F4E037
:101E10000E9409330E947E33FF27EDE0A2E0B4E088
:101E20000E944C36A0EEB6E0AF93BF93E2E0F4E040
:101E30000E9409330E944D3011E001E0BF91AF9143
:101E40000E948935E0EEF6E0ABE3B1E00E94473650
:101E500081E08093620081E0809363008827809313
:101E60006400E6E9F2E70E94CF2FABE3B1E00E9405
:101E7000C92FE6EAF2E70E94CF2F80E08A9380E044
:101E80008A9380E58A9380E08A9381E08A930E9416
:101E90001A3280E08A9387E38A9380E58A9387E306
:101EA0008A9381E08A930E941A328EE48A9387E3B0
:101EB0008A938EE48A9380E08A9381E08A930E94D9
:101EC0001A32EBE3F4E0D190E080FF2400270E9477
:101ED0002D330E946333E6E4F0E70E9466340E94EB
:101EE0000534FF27EDE0A2E0B4E00E944C36EAE4BE
:101EF000F0E70E946F34E2E0F4E00E9409330E94B0
:101F00007E33FF27EDE0A2E0B4E00E944C3687E389
:101F100080933E0480E08093500106B347E00423A1
:101F2000A5E6B0E00C9300916500053011F00C942B
:101F30009F0F8AEF90E00E943E300C94F20585E0FE
:101F400090E00E943E3087E4806487B90E94A63208
:101F5000ABE2B4E08D939C93E2E4F0E70E946F342F
:101F6000EBE2F4E0D190E080FF2400270E942D33C3
:101F70000E94D433FF27EDE0AAE7B0E00E944C3680
:101F8000ABE3B4E04D915C91ABE2B4E00D911C91F8
:101F90000417150710F00C94D50FABE3B4E08D9146
:101FA0009C91ABE2B4E08D939C93ABE2B4E00D91D5
:101FB0001C91ABE3B4E04D915C91041B150BABE2BB
:101FC000B4E00D931C93E2E0F4E00E940E33EBE2E8
:101FD000F4E0D190E080FF2400270E942D330E947E
:101FE0007E33FF27EDE0ADE2B4E00E944C36EDE237
:101FF000F4E00E943037FF27EDE00E94CB32ADE3E2
:10200000B4E0DC9280913D0480933F0406E340916C
:102010003D04041BADE3B4E00C9340913D040091FA
:102020003E04041711F40C94691040913E04009191
:102030003D04041710F00C94441080913E048093EA
:1020400096004091960000913D04041718F011F09D
:102050000C94421080E18A93A6E9B0E08C918A93B7
:102060008EE38A93A6E9B0E08C918A9381E08A930B
:102070000E941A328091960081508093960010F051
:102080000C9421100C94691080913E04809396006A
:1020900040913D0400919600041718F011F00C9443
:1020A000691080E18A93A6E9B0E08C918A938EE36F
:1020B0008A93A6E9B0E08C918A9380E08A930E948B
:1020C0001A32A6E9B0E08C918F5F8C9310F40C94D7
:1020D000481080913D0480933E04EEEFF3E00E94AF
:1020E0000E33EAE7F0E00E9409330E940534FF272F
:1020F000EDE0AAE7B0E00E944C36EAE2F0E70E9489
:102100006F34EAE7F0E00E9409330E947E33FF2734
:10211000EDE0AAE7B0E00E944C36A8E6B0E0EAE2C3
:10212000F0E70E946235E8E6F0E0AAE7B0E00E943E
:10213000E337FF27EDE0AAE7B0E00E944C36EAE77C
:10214000F0E00E940E33E0E4F4E0D190E080FF2460
:1021500000270E942D330E94D433FF27EDE0AAE729
:10216000B0E00E944C368AE090E00E943E30009140
:1021700050010D3211F00C94BB1180E0809350019E
:1021800088E08093620081E08093630088278093D9
:102190006400E4E8F2E70E94CF2FEAE7F0E00E9453
:1021A0000538FF27EDE0A8E6B0E00E944C36E8E6EF
:1021B000F0E00E940E33EAE2F0E70E9466340E94EB
:1021C000D433FF27EDE0A8E6B0E00E944C36A0EE45
:1021D000B6E0AF93BF93E8E6F0E00E9409330E94B7
:1021E0004D3011E001E0BF91AF910E948935E0EEE2
:1021F000F6E0A4E3B1E00E944736EAE7F0E00E948F
:102200000933E2E3F0E70E946F340E94783410F063
:102210000C947C11EAE7F0E00E940933E6E2F0E773
:102220000E946F340E94783418F011F00C941A1147
:102230000C944B11A0EEB6E0AF93BF93EAE7F0E049
:102240000E9409330E944D3011E001E0BF91AF912F
:102250000E948935E0EEF6E0ABE3B1E00E9447363C
:1022600088E08093620081E08093630088278093F8
:102270006400ABE3B1E00E94C92FEAEAF2E70E94F2
:10228000CF2FA4E3B1E00E94C92FEEEAF2E70E944B
:10229000CF2F0C947A11A0EEB6E0AF93BF93EAE78C
:1022A000F0E00E9409330E944D3011E003E0BF913D
:1022B000AF910E948935E0EEF6E0ABE3B1E00E9419
:1022C000473688E08093620081E08093630088272E
:1022D00080936400ABE3B1E00E94C92FEAEAF2E721
:1022E0000E94CF2FA4E3B1E00E94C92FEEEAF2E7EB
:1022F0000E94CF2F0C94BB11E2E3F0E70E946F34F1
:10230000EAE7F0E00E9409330E947E33FF27EDE008
:10231000AAE7B0E00E944C36A0EEB6E0AF93BF93C0
:10232000EAE7F0E00E9409330E944D3011E001E03D
:10233000BF91AF910E948935E0EEF6E0ABE3B1E0EA
:102340000E94473688E08093620081E080936300BA
:10235000882780936400ABE3B1E00E94C92FE6EACE
:10236000F2E70E94CF2FA4E3B1E00E94C92FEEEA6A
:10237000F2E70E94CF2FA0E5B1E08C918F5F8C93A4
:102380000C948D0F0C945D12063011F00C94F11129
:1023900081E08093620081E08093630088278093CE
:1023A0006400E2E8F1E70E94CF2F83E080936200AF
:1023B00081E080936300882780936400E4E9F1E77B
:1023C0000E94CF2F85E08093620081E080936300BC
:1023D000882780936400E6EAF1E70E94CF2F0C94EF
:1023E0005D12073011F00C945D1281E08093620061
:1023F00081E080936300882780936400E2EBF2E73A
:102400000E94CF2F82E08093620081E0809363007E
:10241000882780936400E4ECF2E70E94CF2F83E0EA
:102420008093620081E0809363008827809364003A
:10243000E6EDF2E70E94CF2F84E08093620081E016
:1024400080936300882780936400E8EEF2E70E949F
:10245000CF2F85E08093620081E08093630088271E
:1024600080936400EAEFF2E70E94CF2F86E080932A
:10247000620081E080936300882780936400ECE031
:10248000F3E70E94CF2F87E08093620081E0809382
:102490006300882780936400EEE1F3E70E94CF2F6A
:1024A00088E08093620081E08093630088278093B6
:1024B0006400E0E3F3E70E94CF2F06B347E0042374
:1024C000A5E6B0E00C9300916500053011F00C9486
:1024D0006B120C946F120E946E2F0C945D120E946E
:1024E0001C2180E080935001009150010F3718F0BB
:1024F00011F00C94A21280E3809396000091960054
:102500000A3318F011F00C949612A0E5B1E04C914A
:10251000A6E9B0E05C9191E00E94F331A6E9B0E059
:102520008C918F5F8C9310F40C947E128AE090E073
:102530000E943E30A0E5B1E08C918F5F8C9310F447
:102540000C947412A3E5B2E0E0E8F0E00E949B3640
:10255000A8EDB3E00D931C930E94963100914F01BA
:10256000023011F00C94EA1281E08093620081E065
:1025700080936300882780936400E2E4F3E70E947D
:10258000CF2F83E08093620081E0809363008827EF
:1025900080936400E4E5F3E70E94CF2F84E080930A
:1025A000620081E080936300882780936400E6E600
:1025B000F3E70E94CF2F86E08093620081E0809352
:1025C0006300882780936400E6EAF1E70E94CF2F3A
:1025D0000C944F13063011F00C94171381E0809384
:1025E000620081E080936300882780936400E2E8C2
:1025F000F1E70E94CF2F83E08093620081E0809317
:102600006300882780936400E8E7F3E70E94CF2FF8
:1026100085E08093620081E0809363008827809347
:102620006400E6EAF1E70E94CF2F0C944F130730C5
:1026300011F00C944F1381E08093620081E080934D
:102640006300882780936400EAE8F3E70E94CF2FB5
:1026500083E08093620081E0809363008827809309
:102660006400ECE9F3E70E94CF2F84E080936200DE
:1026700081E080936300882780936400EEE1F3E7B4
:102680000E94CF2F86E08093620081E080936300F8
:10269000882780936400E6EAF1E70E94CF2F06B313
:1026A00047E00423A5E6B0E00C93009165000530F7
:1026B00011F00C945D130C9461130E946E2F0C9416
:1026C0004F130E941C2180E0809350010091500123
:1026D0000F3718F011F00C94941380E38093960058
:1026E000009196000A3318F011F00C948813A0E5BD
:1026F000B1E04C91A6E9B0E05C9191E00E94F33129
:10270000A6E9B0E08C918F5F8C9310F40C94701359
:102710008AE090E00E943E30A0E5B1E08C918F5FAE
:102720008C9310F40C9466130E94963100914F0123
:10273000023011F00C94C51381E08093620081E0B7
:1027400080936300882780936400EEEAF3E70E9499
:10275000CF2F83E08093620081E08093630088271D
:1027600080936400EEEBF3E70E94CF2F84E0809328
:10277000620081E080936300882780936400EEEC20
:10278000F3E70E94CF2F0C941D14063011F00C9427
:10279000F21381E08093620081E0809363008827D8
:1027A00080936400EEEAF3E70E94CF2F83E08093EA
:1027B000620081E080936300882780936400EEEDDF
:1027C000F3E70E94CF2F84E08093620081E0809342
:1027D0006300882780936400ECEEF3E70E94CF2F1C
:1027E0000C941D14073011F00C941D1481E080939B
:1027F000620081E080936300882780936400EEEAA2
:10280000F3E70E94CF2F83E08093620081E0809302
:102810006300882780936400EEEDF3E70E94CF2FDA
:1028200084E08093620081E0809363008827809336
:102830006400ECEEF3E70E94CF2FE2E0F0E00E94AC
:10284000D62FA3E5B2E0E0E8F0E00E948F36A6EDD7
:10285000B3E00D931C930E94963181E08093620057
:1028600081E080936300882780936400EEEAF3E7B9
:102870000E94CF2F85E08093620081E08093630007
:10288000882780936400EAEFF0E70E94CF2F86E06C
:102890008093620081E080936300882780936400C6
:1028A000EAEFF3E70E94CF2FA0EEB6E0E8EDF3E009
:1028B0000E94EE350E94C72F87E08093620081E07E
:1028C00080936300882780936400E2E0F4E70E942D
:1028D000CF2FA0EEB6E0E6EDF3E00E94EE350E94C9
:1028E000C72FA6EDB3E00D911C91A8EDB3E04D917B
:1028F0005C91041B150BA4EEB3E00D931C93E2E472
:10290000F0E70E946F34E4EEF3E0D190E080FF2422
:1029100000270E942D330E94D433FF27EDE0ACED59
:10292000B3E00E944C36EEE4F0E70E946F34E4EE30
:10293000F3E0D190E080FF2400270E942D330E9415
:102940007E33FF27EDE0A6EEB3E00E944C36EEE4C6
:10295000F0E70E946F34ECEDF3E00E9409330E942F
:102960007E33FF27EDE0A0EEB3E00E944C3688E016
:102970008093620081E080936300882780936400E5
:10298000EAE0F4E70E94CF2FECEDF3E00E9430374D
:10299000DD2CEE2CFF2C002FA0EEB6E0FF27EDE0A3
:1029A0000E9409330E944D300E94C72FE2E1F4E7F4
:1029B0000E94CF2FE2E0F0E00E94D62F00914F015D
:1029C000053011F00C94891580E890E0A0E4B4E0A3
:1029D0008D939C93ACECB0E00D911D912D913C91A9
:1029E000A8ECB0E04D915D916D917C910E94D6353F
:1029F000AEEEB0E00D931D932D933D93A0E4B4E0B3
:102A00000D911C912227332749EF54E160E070E0DB
:102A10000E948332A7E3B4E00D931D932D933D9361
:102A2000AEEEB0E04D915D916D917C91A7E3B4E085
:102A30000D911D912D913C910E94DB351CF011F000
:102A40000C94421502E010E0A0E4B4E04D915C91DA
:102A50000E947932A0E4B4E00D931C93A0E4B4E0AA
:102A60000D911C912227332749EF54E160E070E07B
:102A70000E948332A7E3B4E00D931D932D933D9301
:102A80000C941015AEEEB0E00D911D912D913C917E
:102A9000A0E4B4E04D915C91662777270E94E12F76
:102AA000A7E3B4E04D935D936D937D93A0E4B4E010
:102AB0000D911C9140E850E00E94AD2FABE3B4E0D3
:102AC0004D935C93ABE3B4E00D911C91013050E069
:102AD000150718F011F00C946F150C947D15ABE3ED
:102AE000B4E00D911C9142E050E00E94AD2FABE2AA
:102AF000B4E04D935C930C948515ABE3B4E08D91F9
:102B00009C91ABE2B4E08D939C93A1E3B4E00E946E
:102B10006A350E94963187E090E0AEEEB3E08D9387
:102B20009C93AAEEB3E00E946A3580E08093500146
:102B30008091E8008B7F8093E80006B347E0042390
:102B4000A5E6B0E00C93A0E5B1E08C918F5F8C938B
:102B5000009150010F3718F011F00C94B1150C943E
:102B6000631980E080935001A8EEB0E08C9182FB65
:102B700016F00C94C2158091E8008B7F8093E800DA
:102B80000E949631AAEEB3E08C918A9380E08A93FA
:102B9000AAEEB3E08C918A938FE38A9381E08A93C3
:102BA0000E941A3280E08A93AEEEB3E08C918A9351
:102BB0008FE78A93AEEEB3E08C918A9381E08A939B
:102BC0000E941A320E94C82D00914F01053011F069
:102BD0000C94121681E08093620081E08093630080
:102BE000882780936400E4E8F2E70E94CF2F81E019
:102BF0008093620081E08093630088278093640063
:102C0000A4E3B1E00E94C92FE6E1F4E70E94CF2FD0
:102C1000A5EFB3E00E94C92FEAE1F4E70E94CF2FAD
:102C20000C94381688E08093620081E08093630002
:102C3000882780936400E4E8F2E70E94CF2F88E0C1
:102C40008093620081E08093630088278093640012
:102C5000A4E3B1E00E94C92FE6E1F4E70E94CF2F80
:102C6000A5EFB3E00E94C92FEAE1F4E70E94CF2F5D
:102C700000914F01073011F00C94F6168091E80096
:102C800080648093E800E1EFF3E00E940933E2E51D
:102C9000F0E70E946F340E94783410F40C945816B8
:102CA000A4E3B1E0EEE1F4E70E94A0320C94D81660
:102CB000A5EFB3E00E948E34FF27EDE0AEEFB3E066
:102CC0000E944C36E6E5F0E70E946F34EEEFF3E049
:102CD0000E9409330E94D433FF27EDE0AEEFB3E04A
:102CE0000E944C36EAE5F0E70E946F34EEEFF3E025
:102CF0000E9409330E947E33FF27EDE0AEEFB3E080
:102D00000E944C36EEEFF3E00E940E33EAE2F0E769
:102D10000E9466340E94D037FF27EDE0A2E0B4E0C5
:102D20000E944C36E6E2F0E70E946F34E2E0F4E005
:102D30000E9409330E941434FF27EDE0AEEFB3E0A8
:102D40000E944C36E6E2F0E70E946F34E2E0F4E0E5
:102D50000E9409330E940534FF27EDE0A2E0B4E0B1
:102D60000E944C36E2E0F4E00E940E33EEEFF3E016
:102D70000E9409330E947E33FF27EDE0AEEFB3E0FF
:102D80000E944C36A0EEB6E0AF93BF93EEEFF3E0B7
:102D90000E9409330E944D3011E002E0BF91AF91D3
:102DA0000E948935E0EEF6E0A4E3B1E00E944736E8
:102DB00081E08093620081E08093630088278093A4
:102DC0006400E4E8F2E70E94CF2F81E08093620084
:102DD00081E080936300882780936400E2E2F4E757
:102DE0000E94CF2FA4E3B1E00E94C92F00914F01B0
:102DF000023011F00C945A19A3E5B1E0E0E8F0E0DC
:102E00000E94A736ABE2B4E00D931C93A3E3B4E0B9
:102E10004D935C9387E08093620081E08093630030
:102E2000882780936400EEE2F4E70E94CF2FA0EEA3
:102E3000B6E0EBE2F4E00E94EE350E94C72F86E098
:102E40008093620081E08093630088278093640010
:102E5000E4E3F4E70E94CF2FA0EEB6E0E3E3F4E072
:102E60000E94EE350E94C72FABE2B4E00D911C9199
:102E70004FE050E0040F151FA1E3B4E00D931C9345
:102E800080913304809396004091960001E00417EE
:102E900018F011F00C946E17A1E3B4E04D915C9121
:102EA000A6E9B0E0AD90BB24A1E5B1E0AA0CBB1C43
:102EB000AA0DBB1D0D911C910417150718F011F0F8
:102EC0000C9464170C9466170C946E1780919600FE
:102ED00081508093960010F00C94441780919600D6
:102EE000809335048091330480939600009196007E
:102EF0000F3718F011F00C949F17A1E3B4E04D9137
:102F00005C91A6E9B0E0AD90BB24A1E5B1E0AA0CCC
:102F1000BB1CAA0DBB1D0D911C910417150718F0C1
:102F200011F00C9495170C9497170C949F17A6E921
:102F3000B0E08C918F5F8C9310F40C947617809195
:102F4000960080933604A6E3B4E00C911127222763
:102F50003327A5E3B4E04C915527662777270E94D5
:102F6000D635A7E3B4E00D931D932D933D93A7E3CE
:102F7000B4E00D911D912D913C91A0E7B0E04D91F1
:102F80005D916D917C910E948332A7E3B4E00D9333
:102F90001D932D933D930091360440913504040F09
:102FA000A5E3B4E00C93A5E3B4E00C9142E00E94E9
:102FB0007F360C93E3E3F4E0D190E080FF24002718
:102FC0000E942D330E9463332F933F934F935F935F
:102FD000E0E7F0E00E9409330E942D335F914F91AA
:102FE0003F912F910E94D433FF27EDE0A7E2B4E098
:102FF0000E944C36E7E2F4E00E940E33E8ECF0E089
:103000000E9409330E942D330E941434FF27EDE003
:10301000A7E2B4E00E944C36E2E9F0E00E940933F6
:103020000E942D330E946333E7E2F4E00E940933EB
:103030000E947E33FF27EDE0ABE4B1E00E944C3606
:10304000A0EEB6E0AF93BF93EBE4F1E00E9409334A
:103050000E944D3011E005E0BF91AF910E9489358B
:10306000E0EEF6E0A4E3B1E00E94473687E080930B
:10307000620081E080936300882780936400EAE324
:10308000F4E70E94CF2FA4E3B1E00E94C92FEEE342
:10309000F4E70E94CF2FE2E9F0E00E9409330E949A
:1030A0002D330E9463332F933F934F935F93E7E356
:1030B000F4E00E9409330E942D335F914F913F91BC
:1030C0002F910E947E33FF27EDE0A7E2B4E00E943B
:1030D0004C36E7E2F4E00E940E33EBE4F1E00E94AC
:1030E00009330E947E33FF27EDE0A7E2B4E00E949F
:1030F0004C36E7E2F4E00E943037FF27EDE0A7E22C
:10310000B4E00E944C3684E08093620081E08093BA
:103110006300882780936400E2E4F4E70E94CF2FE5
:10312000A0EEB6E0E7E2F4E00E9409330E944D30E1
:103130000E94C72FEBE4F1E00E940E33EBE4F1E0D4
:103140000E9409330E94D433FF27EDE0ABE4B1E0E5
:103150000E944C36EEE5F0E70E946F34EBE4F1E0BC
:103160000E9409330E94D433FF27EDE0ABE4B1E0C5
:103170000E944C36EEE1F4E00E940E33EBE4F1E005
:103180000E9409330E94D433FF27EDE0A7E2B4E0A8
:103190000E944C36E2E6F0E70E946F34E7E2F4E08A
:1031A0000E9409330E94D433FF27EDE0A7E2B4E088
:1031B0000E944C36E7E2F4E00E940E33E6E2F0E7CC
:1031C0000E9466340E947E33FF27EDE0A7E2B4E060
:1031D0000E944C36A0EEB6E0AF93BF93E7E2F4E076
:1031E0000E9409330E944D3011E001E0BF91AF9180
:1031F0000E948935E0EEF6E0A4E3B1E00E94473694
:1032000085E08093620081E080936300882780934B
:103210006400E6E4F4E70E94CF2FA4E3B1E00E944B
:10322000C92FEAE4F4E70E94CF2FEAE1F4E00E941C
:103230000E33EBE4F1E00E9409330E94D433FF2700
:10324000EDE0A7E2B4E00E944C36E7E2F4E00E9431
:103250000E33E6E6F0E70E9466340E947E33FF27D5
:10326000EDE0A7E2B4E00E944C36E7E2F4E00E9411
:103270003037FF27EDE0A7E2B4E00E944C3686E04D
:103280008093620081E080936300882780936400CC
:10329000EEE4F4E70E94CF2FA0EEB6E0E7E2F4E020
:1032A0000E9409330E944D300E94C72FE2E5F4E7E7
:1032B0000E94CF2FA8EEB0E08C9185FB16F00C9405
:1032C00063190E94C82D00914F01053011F40C9430
:1032D000021A41E050E060E070E0A8EDB0E00D912E
:1032E0001D912D913C910E94DB3511F00C94AC198D
:1032F000EAEEF0E00E9409330E942D330E9463330E
:103300002F933F934F935F93E0E5F1E0D080EE245D
:10331000FF2400270E942D335F914F913F912F9101
:103320000E94D433FF27EDE0AEEFB0E00E944C36B0
:10333000EEEFF0E00E940E33E8ECF0E00E9409337B
:103340000E942D330E941434FF27EDE0AEEFB0E071
:103350000E944C360C94EC19E0E5F1E0D080EE24AC
:10336000FF2400270E942D330E946333E2EFF0E038
:103370000E9409330E94D433FF27EDE0AAEFB0E0AA
:103380000E944C36E6EFF0E00E940E33EAEFF0E0E8
:103390000E9409330E941434FF27EDE0AAEFB0E049
:1033A0000E944C36EAEFF0E00E940E33EAE2F0E7CA
:1033B0000E9466340E94D037FF27EDE0AAEFB0E00C
:1033C0000E944C36EAEFF0E00E943037FF27EDE034
:1033D000AEEFB0E00E944C360E949E220091500158
:1033E000003011F00C94FA1985E090E00E943E3014
:1033F0000C94021AEF93FF93ECE8F1E00E94353051
:10340000FF91EF910091500141E0040FA1E5B1E07F
:103410000C9300914F01053011F00C944D1B00915D
:103420005001013081E008F480E08F930091500159
:103430000E3781E010F009F080E09F918923882306
:1034400011F40C94B31AA1E5B1E0AD90BB24A1E551
:10345000B1E0AA0CBB1CAA0DBB1D0E946A3581E01D
:1034600080939600ABE3B4E04D915C91A6E9B0E0A7
:103470000D9111270417150718F011F00C94B11ACB
:10348000E7E3F4E00E9409330E942D330E94633386
:103490002F933F934F935F93E1E3F4E0D190E0806B
:1034A000FF2400270E942D335F914F913F912F9170
:1034B0000E94D433FF27EDE0AEEFB0E00E944C361F
:1034C000EEEFF0E00E940E33E8ECF0E00E940933EA
:1034D0000E942D330E941434FF27EDE0AEEFB0E0E0
:1034E0000E944C360E949E22A1E3B4E00E947B2FF2
:1034F00087E4806487B90E94A632A0E4B4E08D938B
:103500009C93A1E5B1E0AD90BB24A1E5B1E0AA0C8C
:10351000BB1CAA0DBB1D4D915C91A0E4B4E00D91C4
:103520001C910417150718F011F00C94991A0C94BB
:10353000A91AA0E4B4E08D919C91A1E5B1E0AD9011
:10354000BB24A1E5B1E0AA0CBB1CAA0DBB1D8D9349
:103550009C93A6E9B0E08C918F5F8C9310F40C944F
:10356000321A0C944B1BA1E5B1E0AD90BB24A1E550
:10357000B1E0AA0CBB1CAA0DBB1D0E946A3581E0FC
:1035800080939600ABE2B4E04D915C91A6E9B0E087
:103590000D9111270417150718F011F00C94411B19
:1035A000E7E3F4E00E9409330E942D330E94633365
:1035B0002F933F934F935F93E1E3F4E0D190E0804A
:1035C000FF2400270E942D335F914F913F912F914F
:1035D0000E94D433FF27EDE0AEEFB0E00E944C36FE
:1035E000EEEFF0E00E940E33E8ECF0E00E940933C9
:1035F0000E942D330E941434FF27EDE0AEEFB0E0BF
:103600000E944C360E949E22A1E3B4E00E947B2FD0
:1036100087E4806487B90E94A632A0E4B4E08D9369
:103620009C93A1E5B1E0AD90BB24A1E5B1E0AA0C6B
:10363000BB1CAA0DBB1D4D915C91A0E4B4E00D91A3
:103640001C910417150718F011F00C94291B0C9409
:10365000391BA0E4B4E08D919C91A1E5B1E0AD905F
:10366000BB24A1E5B1E0AA0CBB1CAA0DBB1D8D9328
:103670009C93A6E9B0E08C918F5F8C9310F40C942E
:10368000C21A009150010F3711F00C944B1BA1E3AB
:10369000B4E00E946A350C945E1B87E4806487B9AD
:1036A0000E94A632A1E5B1E0AD90BB24A1E5B1E056
:1036B000AA0CBB1CAA0DBB1D8D939C93A1E5B1E088
:1036C000AD90BB24A1E5B2E0AA0CBB1CAA0DBB1DAA
:1036D0004D915C91A1E5B1E0AD90BB24A1E5B1E0D5
:1036E000AA0CBB1CAA0DBB1D0D911C91041715073C
:1036F00018F011F00C947E1B0C94961BA1E5B1E020
:10370000AD90BB24A1E5B2E0AA0CBB1CAA0DBB1D69
:103710008D919C91A1E5B1E0AD90BB24A1E5B1E014
:10372000AA0CBB1CAA0DBB1D8D939C93A8EDB3E006
:103730004D915C91A1E5B1E0AD90BB24A1E5B1E074
:10374000AA0CBB1CAA0DBB1D0D911C9104171507DB
:1037500010F00C94BB1BA8EDB3E08D919C91A1E5FA
:10376000B1E0AD90BB24A1E5B1E0AA0CBB1CAA0D51
:10377000BB1D8D939C93A1E5B1E0AD90BB24A1E569
:10378000B2E0AA0CBB1CAA0DBB1D0D911C91A1E5BA
:10379000B1E0AD90BB24A1E5B1E0AA0CBB1CAA0D21
:1037A000BB1D4D915C91041B150BAAEFB3E00D936B
:1037B0001C93E6EEF3E00E940E33EAEFF3E0D190C3
:1037C000E080FF2400270E942D330E947E33FF27D4
:1037D000EDE0ABE4B1E00E944C36EBE4F1E00E9496
:1037E0003037FF27EDE00E94CB32AAEFB3E0DD9245
:1037F000EC92AAEFB3E00D911C9147E050E0040F6A
:10380000151FAAEFB3E00D931C93AAEFB3E00D913F
:103810001C91003050E0150710F00C94131CAAEF17
:10382000B3E00E946A35AAEFB3E00D911C910F330B
:1038300050E0150718F011F00C94201C0C94261C75
:103840008FE390E0AAEFB3E08D939C9300914F013A
:10385000053011F00C945F1C0FE740915001041BE0
:10386000A2E5B1E00C93A2E5B1E08C918A938FE3DD
:103870008A93A2E5B1E08C918A93A1E5B1E0AD9085
:10388000BB24A2E5B3E0AA0DBB1D8C918A9380E016
:103890008A930E941A32A2E5B1E08C918A938FE359
:1038A0008A93A2E5B1E08C918A93AAEFB3E08C9160
:1038B0008A9381E08A930E941A320C94771CA0E5C7
:1038C000B1E04C91A1E5B1E0AD90BB24A2E5B3E03D
:1038D000AA0DBB1D5C9190E00E94F331A0E5B1E020
:1038E0004C91AAEFB3E05C9191E00E94F33180919A
:1038F000FA03A1E5B1E0AD90BB24A2E5B3E0AA0DC7
:10390000BB1D8C9300916500053011F00C94901C48
:103910000E946E2F8AEF90E00E943E300C94F205D8
:1039200000916500033011F00C940A1E0E946E2F66
:10393000AAEEB3E08C918A9380E08A93AAEEB3E07A
:103940008C918A938FE38A9380E08A930E941A3243
:10395000AAEEB3E00E94812FAAEEB3E00D911C9174
:10396000003050E015070CF402C00C94361DAAEE8E
:10397000B3E00E946A358091E80084608093E8009B
:10398000ACECB0E00D911D912D913C91A8ECB0E014
:103990004D915D916D917C910E94D635ACE6B0E081
:1039A0000D931D932D933D93ACE6B0E00D911D91C9
:1039B0002D913C914AE050E060E070E00E94E12FE0
:1039C000ACE6B0E04D935D936D937D93A8ECB0E0D1
:1039D0000D911D912D913C91ACE6B0E04D915D9122
:1039E0006D917C910E94D635A8ECB0E00D931D93AB
:1039F0002D933D93A0ECB0E04D915D916D917C9144
:103A0000A8ECB0E00D911D912D913C910E94DB3509
:103A10000CF402C00C94221DA8ECB0E00D911D9195
:103A20002D913C91ACE6B0E04D915D916D917C9112
:103A30000E94D135A8ECB0E00D931D932D933D93DA
:103A40000C94361DACECB0E00D911D912D913C9184
:103A5000ACE6B0E04D915D916D917C910E94D635C0
:103A6000ACECB0E00D931D932D933D93AAEEB3E023
:103A70008C918A9380E08A93AAEEB3E08C918A932A
:103A80008FE38A9381E08A930E941A3280E08A93BE
:103A9000AEEEB3E08C918A938FE78A93AEEEB3E0FB
:103AA0008C918A9381E08A930E941A3200914F018F
:103AB000053011F40C947D1D80E08093F00300919B
:103AC000F0030F3718F011F00C947D1DA0EFB3E058
:103AD0004C91A0EFB3E0AD90BB24A3E5B3E0AA0DF9
:103AE000BB1D5C9191E00E94F331A0EFB3E08C919B
:103AF0008F5F8C9310F40C945F1D00914F01053083
:103B000011F00C94B51DEAEEF0E00E9409330E941A
:103B10002D330E9463332F933F934F935F93E2E5DE
:103B2000F1E0D080EE24FF2400270E942D335F9126
:103B30004F913F912F910E94D433FF27EDE0AEEFDC
:103B4000B0E00E944C36EEEFF0E00E940E33E8EC5D
:103B5000F0E00E9409330E942D330E941434FF27A5
:103B6000EDE0AEEFB0E00E944C360E94C82D00910F
:103B70004F01053011F00C94D81D81E08093620054
:103B800081E080936300882780936400A4E3B1E020
:103B90000E94C92FE6E5F4E70E94CF2FA5EFB3E01E
:103BA0000E94C92FEAE1F4E70E94CF2F0C94F11D87
:103BB00088E08093620081E080936300882780938F
:103BC0006400A4E3B1E00E94C92FE6E5F4E70E9497
:103BD000CF2FA5EFB3E00E94C92FEAE1F4E70E94DE
:103BE000CF2F84E690E00E943E3006B347E00423E6
:103BF000A5E6B0E00C9300916500033011F00C9441
:103C0000051E0E946E2F0C94981C8091E800806223
:103C10008093E80000916500013011F00C94881F3A
:103C20000E946E2FAAEEB3E08C918A9380E08A9373
:103C3000AAEEB3E08C918A938FE38A9380E08A9313
:103C40000E941A32AAEEB3E00E947B2FAAEEB3E0E4
:103C50000D911C910F3750E015071CF011F00C94DA
:103C6000331E0C94B61E8FE790E0AAEEB3E08D935E
:103C70009C938091E80084608093E800ACECB0E015
:103C80000D911D912D913C91A8ECB0E04D915D916D
:103C90006D917C910E94D635ACE6B0E00D931D93FA
:103CA0002D933D93ACE6B0E00D911D912D913C918B
:103CB0004AE050E060E070E00E94E12FACE6B0E046
:103CC0004D935D936D937D93ACECB0E00D911D91A0
:103CD0002D913C91ACE6B0E04D915D916D917C9160
:103CE0000E94D135ACECB0E00D931D932D933D9324
:103CF000ACEBB0E04D915D916D917C91ACECB0E09E
:103D00000D911D912D913C910E94DB351CF011F01D
:103D10000C948C1E0C94A21EACECB0E00D911D9185
:103D20002D913C91ACE6B0E04D915D916D917C910F
:103D30000E94D635ACECB0E00D931D932D933D93CE
:103D40000C94B61EA8ECB0E00D911D912D913C9104
:103D5000ACE6B0E04D915D916D917C910E94D135C2
:103D6000A8ECB0E00D931D932D933D93AAEEB3E024
:103D70008C918A9380E08A93AAEEB3E08C918A9327
:103D80008FE38A9381E08A930E941A3280E08A93BB
:103D9000AEEEB3E08C918A938FE78A93AEEEB3E0F8
:103DA0008C918A9381E08A930E941A3200914F018C
:103DB000053011F40C94FD1E80E08093F003009117
:103DC000F0030F3718F011F00C94FD1EA0EFB3E0D4
:103DD0004C91A0EFB3E0AD90BB24A3E5B3E0AA0DF6
:103DE000BB1D5C9191E00E94F331A0EFB3E08C9198
:103DF0008F5F8C9310F40C94DF1E00914F010530FF
:103E000011F00C94351FEAEEF0E00E9409330E9495
:103E10002D330E9463332F933F934F935F93E2E5DB
:103E2000F1E0D080EE24FF2400270E942D335F9123
:103E30004F913F912F910E94D433FF27EDE0AEEFD9
:103E4000B0E00E944C36EEEFF0E00E940E33E8EC5A
:103E5000F0E00E9409330E942D330E941434FF27A2
:103E6000EDE0AEEFB0E00E944C360E94C82D00910C
:103E70004F01053011F00C94581F81E080936200CF
:103E800081E080936300882780936400A4E3B1E01D
:103E90000E94C92FE6E5F4E70E94CF2FA5EFB3E01B
:103EA0000E94C92FEAE1F4E70E94CF2F0C94711F02
:103EB00088E08093620081E080936300882780938C
:103EC0006400A4E3B1E00E94C92FE6E5F4E70E9494
:103ED000CF2FA5EFB3E00E94C92FEAE1F4E70E94DB
:103EE000CF2F84E690E00E943E3006B347E00423E3
:103EF000A5E6B0E00C9300916500013011F00C9440
:103F0000831F0C94121E8091E80080628093E80069
:103F100000916500043011F00C9451200E946E2F26
:103F200080E08A93AEEEB3E08C918A938FE78A9318
:103F3000AEEEB3E08C918A9380E08A930E941A32AD
:103F4000AEEEB3E00E947B2FAEEEB3E00D911C917C
:103F50000F3350E015071CF011F00C94B11F0C94B6
:103F6000B71F8FE390E0AEEEB3E08D939C9380E0BB
:103F70008A93AEEEB3E08C918A938FE78A93AEEE8C
:103F8000B3E08C918A9381E08A930E941A32AAEE60
:103F9000B3E08C918A9380E08A93AAEEB3E08C918F
:103FA0008A938FE38A9381E08A930E941A32009168
:103FB0004F01053011F40C94FE1F80E08093F00354
:103FC0000091F0030F3718F011F00C94FE1FA0EFD2
:103FD000B3E04C91A0EFB3E0AD90BB24A3E5B3E018
:103FE000AA0DBB1D5C9191E00E94F331A0EFB3E0FC
:103FF0008C918F5F8C9310F40C94E01F0E94C82D5D
:1040000000914F01053011F00C94212081E0809344
:10401000620081E080936300882780936400A4E3BA
:10402000B1E00E94C92FE6E5F4E70E94CF2FA5EF8B
:10403000B3E00E94C92FEAE1F4E70E94CF2F0C946D
:104040003A2088E08093620081E0809363008827B3
:1040500080936400A4E3B1E00E94C92FE6E5F4E791
:104060000E94CF2FA5EFB3E00E94C92FEAE1F4E749
:104070000E94CF2F84E690E00E943E3006B347E0D6
:104080000423A5E6B0E00C9300916500043011F024
:104090000C944C200C94901F8091E80080628093D7
:1040A000E80000916500063011F00C9418210E9480
:1040B0006E2F80E08A93AEEEB3E08C918A938FE707
:1040C0008A93AEEEB3E08C918A9380E08A930E944B
:1040D0001A32AEEEB3E00E94812FAEEEB3E00D9146
:1040E0001C91003050E015070CF402C00C947C20A9
:1040F000AEEEB3E00E946A3580E08A93AEEEB3E0A4
:104100008C918A938FE78A93AEEEB3E08C918A9379
:1041100081E08A930E941A32AAEEB3E08C918A93CE
:1041200080E08A93AAEEB3E08C918A938FE38A931E
:1041300081E08A930E941A3200914F01053011F4F8
:104140000C94C32080E08093F0030091F0030F37BC
:1041500018F011F00C94C320A0EFB3E04C91A0EF45
:10416000B3E0AD90BB24A3E5B3E0AA0DBB1D5C9109
:1041700091E00E94F331A0EFB3E08C918F5F8C93BC
:1041800010F40C94A5200E94C82D00914F01053019
:1041900011F00C94E62081E08093620081E080932E
:1041A0006300882780936400A4E3B1E00E94C92FD4
:1041B000E6E5F4E70E94CF2FA5EFB3E00E94C92FF8
:1041C000EAE1F4E70E94CF2F0C94FF2088E080936F
:1041D000620081E080936300882780936400A4E3F9
:1041E000B1E00E94C92FE6E5F4E70E94CF2FA5EFCA
:1041F000B3E00E94C92FEAE1F4E70E94CF2F84E6E2
:1042000090E00E943E3006B347E00423A5E6B0E00C
:104210000C9300916500063011F00C9413210E945C
:104220006E2F0C9459208091E80080628093E80002
:104230000C949D150C94FF050E94092281E0809347
:10424000420400914204003818F011F00C94CA2185
:1042500041E050E060E070E0A8EDB0E00D911D910C
:104260002D913C910E94DB3511F00C946B21EAEE0C
:10427000F0E00E9409330E942D330E9463332F9394
:104280003F934F935F93E2E4F4E0D080EE24FF2469
:1042900000270E942D335F914F913F912F910E94F3
:1042A000D433FF27EDE0AEEFB0E00E944C36EEEFE6
:1042B000F0E00E940E33E8ECF0E00E9409330E9427
:1042C0002D330E941434FF27EDE0AEEFB0E00E94E2
:1042D0004C360C94AB21E2E4F4E0D080EE24FF24D1
:1042E00000270E942D330E946333E2EFF0E00E942A
:1042F00009330E94D433FF27EDE0AAEFB0E00E941B
:104300004C36E6EFF0E00E940E33EAEFF0E00E9458
:1043100009330E941434FF27EDE0AAEFB0E00E94B9
:104320004C36EAEFF0E00E940E33EAE2F0E70E943A
:1043300066340E94D037FF27EDE0AAEFB0E00E947C
:104340004C36EAEFF0E00E943037FF27EDE0AEEFA9
:10435000B0E00E944C360E949E2281E090E00E94D4
:104360003E3087E4806487B90E94A632A2E4B4E0BC
:10437000AD90BB24A1E5B2E0AA0CBB1CAA0DBB1DED
:104380008D939C93A2E4B4E08C918F5F8C9310F496
:104390000C9421210895A881B9818D919C91A5E467
:1043A000B4E08D939C93939881E0809347040091AF
:1043B0004704003118F011F00C940722A5E4B4E092
:1043C0000D911C9140E050E804231523A3E4B4E0D0
:1043D0000D931C93A3E4B4E00D911C91003050E8C0
:1043E000150711F00C94F721959A0C94F8219598E3
:1043F0009498949A91E0A5E4B4E00E94AF32A7E4C7
:10440000B4E08C918F5F8C9310F40C94D721939A25
:104410000895ACECB0E04D915D916D917C91A8EC6C
:10442000B0E00D911D912D913C910E94DB3511F072
:104430000C942022AEEEB0E00E946C350C949D22CC
:10444000ACECB0E00D911D912D913C91A8ECB0E049
:104450004D915D916D917C910E94D635AAEEB0E0B0
:104460000D931D932D933D93AAEEB0E00D911D91F8
:104470002D913C9140E850E060E070E00E94E12F17
:10448000AAEEB0E04D935D936D937D9342E050E0D2
:1044900060E070E0A8EDB0E00D911D912D913C9190
:1044A0000E94DB3511F00C949D22ECECF0E00E94B0
:1044B00009330E942D33A2EFB0E00E945E33E2EF99
:1044C000F0E00E940538FF27EDE0A2EFB0E00E9487
:1044D0004C36E8ECF0E00E9409330E942D33A6EF41
:1044E000B0E00E945E33E6EFF0E00E940538FF275F
:1044F000EDE0A6EFB0E00E944C36E6EFF0E00E945F
:104500000E33E2EFF0E00E9409330E940534FF27EA
:10451000EDE0A2EFB0E00E944C36EAE6F0E70E9440
:104520006F34E2EFF0E00E9409330E947E33FF27F0
:10453000EDE0A2EFB0E00E944C360895EEEFF0E01F
:104540000E94CB32ACE4B4E0EDE0FF270E944C3691
:10455000ACE4B4E00D911C914FEF5FE3042315230D
:10456000AAE4B4E00D931C9381E080935004009181
:1045700050040E3018F011F00C94CB2291E0ACE412
:10458000B4E00E94BA32A0E5B4E08C918F5F8C93C6
:1045900010F40C94B722ACE4B4E00D911C914FEFF1
:1045A0005FE304231523A8E4B4E00D931C93A8E46F
:1045B000B4E00D911C9140E050E4040F151FA8E4F5
:1045C000B4E00D931C93AAE4B4E00D911C9140E07B
:1045D00050E4040F151FAAE4B4E00D931C935A9203
:1045E0004A92A4E7B0E08D919C91A42DB52D8D93B6
:1045F0009C9382E00E94772F0E94CB21229682E03A
:104600000E94732F5A924A92AAE4B4E08D919C9131
:10461000A42DB52D8D939C9382E00E94772F0E944C
:10462000CB21229682E00E94732F5A924A92A8E4EC
:10463000B4E08D919C91A42DB52D8D939C9382E037
:104640000E94772F0E94CB21229682E00E94732F36
:1046500008950E94963180E0809352048BE080930D
:10466000510481E08093530400912A01023110F03B
:104670000C945B2340912A0100915104041711F01E
:104680000C94452381E080935204A3E5B4E08C911F
:104690008093620081E080936300A2E5B4E08C9196
:1046A00080936400E8E5F4E70E94CF2FA3E5B4E02F
:1046B0008C918F5F8C9380E080935204A1E5B4E0ED
:1046C0008C918F5F8C9300912A01033110F00C9430
:1046D000982340912A0100915104041711F00C9481
:1046E000742381E080935204A3E5B4E08C9180931D
:1046F000620081E080936300A2E5B4E08C91809336
:104700006400E0E6F4E70E94CF2FABE2B1E00D9148
:10471000112746E050E00E947932A0E0B1E0A00FFE
:10472000B11F0E94C92FA3E5B4E08C918F5F8C93D9
:1047300080E080935204A1E5B4E08C918F5F8C936C
:1047400000912A01043110F00C942B2440912A018D
:1047500000915104041711F00C94B12381E080936F
:104760005204E2E9F0E00E9409330E942D330E94D6
:1047700063332F933F934F935F93E8ECF0E00E94F5
:1047800009330E942D335F914F913F912F910E94E9
:104790007E33FF27EDE0ABE4B1E00E944C36A0EEA3
:1047A000B6E0AF93BF93EBE4F1E00E9409330E94BF
:1047B0004D3011E004E0BF91AF910E948935E0EEE9
:1047C000F6E0A4E3B1E00E944736EBE4F1E00E949A
:1047D0000933EAE2F0E70E946F340E94783410F067
:1047E0000C940D24A3E5B4E08C918093620081E0E9
:1047F00080936300A2E5B4E08C9180936400ECE6C2
:10480000F4E70E94CF2FA4E3B1E00E94C92FEEE3AA
:10481000F4E70E94CF2F0C942624A3E5B4E08C91FA
:104820008093620081E080936300A2E5B4E08C9104
:1048300080936400E4E7F4E70E94CF2FA4E3B1E0A3
:104840000E94C92FEEE3F4E70E94CF2FA3E5B4E066
:104850008C918F5F8C9380E080935204A1E5B4E04B
:104860008C918F5F8C9340912A0100915104041721
:1048700011F00C943E2481E080935204E2E9F0E0D0
:104880000E9409330E942D330E9463332F933F937C
:104890004F935F93ECECF0E00E9409330E942D33BC
:1048A0005F914F913F912F910E947E33FF27EDE062
:1048B000ABE4B1E00E944C36A0EEB6E0AF93BF93FC
:1048C000EBE4F1E00E9409330E944D3011E004E076
:1048D000BF91AF910E948935E0EEF6E0A4E3B1E02C
:1048E0000E944736EBE4F1E00E940933EAE2F0E788
:1048F0000E946F340E94783410F00C949A24A3E53F
:10490000B4E08C918093620081E080936300A2E523
:10491000B4E08C9180936400ECE7F4E70E94CF2F21
:10492000A4E3B1E00E94C92FEEE3F4E70E94CF2F89
:104930000C94B324A3E5B4E08C918093620081E0F1
:1049400080936300A2E5B4E08C9180936400E4E876
:10495000F4E70E94CF2FA4E3B1E00E94C92FEEE359
:10496000F4E70E94CF2F80E080935204A1E5B4E0E9
:104970008C918F5F8C93A3E5B4E08C918F5F8C93C7
:1049800040912A0100915104041711F00C94CB249A
:1049900081E08093520441E050E060E070E0A8EDD7
:1049A000B0E00D911D912D913C910E94DB3511F0ED
:1049B0000C94E224A2E4B1E0ECE8F4E70E94A03217
:1049C0000C94E824A2E4B1E0E0E9F4E70E94A0320C
:1049D000A3E5B4E08C918093620081E08093630052
:1049E000A2E5B4E08C9180936400E4E9F4E70E94CE
:1049F000CF2FA2E4B1E00E94C92F80E0809352043F
:104A00000E940922A1E5B4E08C918F5F8C93A3E50D
:104A1000B4E08C918F5F8C9340912A0100915104F6
:104A2000041711F00C94172581E08093520441E0A3
:104A300050E060E070E0A4EDB0E00D911D912D918B
:104A40003C910E94DB3511F00C942E25A2E4B1E0DC
:104A5000E2EAF4E70E94A0320C943425A2E4B1E02B
:104A6000E6EAF4E70E94A032A3E5B4E08C918093DB
:104A7000620081E080936300A2E5B4E08C918093B2
:104A80006400EAEAF4E70E94CF2FA2E4B1E00E94BA
:104A9000C92F80E080935204A1E5B4E08C918F5F30
:104AA0008C93A3E5B4E08C918F5F8C9340912A01A5
:104AB00000915104041711F00C94612581E080935A
:104AC0005204E2E9F0E00E9409330E942D330E9473
:104AD00063332F933F934F935F93E4ECF0E00E9496
:104AE00009330E942D335F914F913F912F910E9486
:104AF0007E33FF27EDE0ABE4B1E00E944C36A0EE40
:104B0000B6E0AF93BF93EBE4F1E00E9409330E945B
:104B10004D3011E004E0BF91AF910E948935E0EE85
:104B2000F6E0A4E3B1E00E944736EBE4F1E00E9436
:104B30000933EAE2F0E70E946F340E94783410F003
:104B40000C94BD25A3E5B4E08C918093620081E0D4
:104B500080936300A2E5B4E08C9180936400E8EB5D
:104B6000F4E70E94CF2FA4E3B1E00E94C92FEEE347
:104B7000F4E70E94CF2F0C94D625A3E5B4E08C91E6
:104B80008093620081E080936300A2E5B4E08C91A1
:104B900080936400E0ECF4E70E94CF2FA4E3B1E03F
:104BA0000E94C92FEEE3F4E70E94CF2F80E08093AC
:104BB0005204A1E5B4E08C918F5F8C93A3E5B4E03F
:104BC0008C918F5F8C9340912A01009151040417BE
:104BD00011F00C94EE2581E080935204009126049C
:104BE000013011F00C940726A3E5B4E08C9180937A
:104BF000620081E080936300A2E5B4E08C91809331
:104C00006400E8ECF4E70E94CF2F0C946126023098
:104C100011F00C941E26A3E5B4E08C918093620001
:104C200081E080936300A2E5B4E08C9180936400FE
:104C3000EAEDF4E70E94CF2F0C946126033011F0C7
:104C40000C943526A3E5B4E08C918093620081E05A
:104C500080936300A2E5B4E08C9180936400ECEE55
:104C6000F4E70E94CF2F0C946126043011F00C94CD
:104C70004C26A3E5B4E08C918093620081E08093A0
:104C80006300A2E5B4E08C9180936400EEEFF4E75A
:104C90000E94CF2F0C946126053011F00C946126F0
:104CA000A3E5B4E08C918093620081E0809363007F
:104CB000A2E5B4E08C9180936400E0E1F5E70E9406
:104CC000CF2F80E080935204A1E5B4E08C918F5FF8
:104CD0008C93A3E5B4E08C918F5F8C9300912A01B3
:104CE000013118F011F00C9477260C94BA274091FA
:104CF0002A0100915104041711F00C94822681E0DE
:104D000080935204A0EEB6E0AF93BF93EAE1F4E0E3
:104D10000E9409330E944D3011E001E0BF91AF9134
:104D20000E948935E0EEF6E0A4E3B1E00E94473648
:104D3000EAE1F4E00E940933EAE2F0E70E946F340E
:104D40000E94783410F00C94C026A3E5B4E08C9156
:104D50008093620081E080936300A2E5B4E08C91CF
:104D600080936400E2E2F5E70E94CF2FA4E3B1E074
:104D70000E94C92FEAE4F4E70E94CF2F0C94B227D7
:104D8000EAE1F4E00E940933EAE2F0E70E946F34BE
:104D90000E94783481E008F480E08F93EAE1F4E047
:104DA0000E940933EEE6F0E70E946F340E947834E7
:104DB00081E010F009F080E09F918923882311F4AD
:104DC0000C94FD26A3E5B4E08C918093620081E011
:104DD00080936300A2E5B4E08C9180936400EEE2DE
:104DE000F5E70E94CF2FA4E3B1E00E94C92FEAE4C7
:104DF000F4E70E94CF2F0C94B227EAE1F4E00E947E
:104E00000933EEE2F0E70E946F340E94783481E0CB
:104E100008F480E08F93EAE1F4E00E940933E2E7CE
:104E2000F0E70E946F340E94783481E010F009F0BE
:104E300080E09F918923882311F40C943A27A3E5FD
:104E4000B4E08C918093620081E080936300A2E5DE
:104E5000B4E08C9180936400EAE3F5E70E94CF2FE1
:104E6000A4E3B1E00E94C92FEAE4F4E70E94CF2F47
:104E70000C94B227EAE1F4E00E940933E2E3F0E7A0
:104E80000E946F340E94783481E008F480E08F93B0
:104E9000EAE1F4E00E940933E6E7F0E70E946F34AC
:104EA0000E94783481E010F009F080E09F9189231E
:104EB000882311F40C947727A3E5B4E08C918093B8
:104EC000620081E080936300A2E5B4E08C9180935E
:104ED0006400E4E4F5E70E94CF2FA4E3B1E00E9470
:104EE000C92FEAE4F4E70E94CF2F0C94B227EAE13D
:104EF000F4E00E940933EAE7F0E70E946F340E9471
:104F0000783481E008F480E08F93EAE1F4E00E94D5
:104F10000933EEE7F0E70E946F340E94783481E0B5
:104F200010F009F080E09F918923882311F40C94FC
:104F3000B227A3E5B4E08C918093620081E0809376
:104F40006300A2E5B4E08C9180936400EEE4F5E7A1
:104F50000E94CF2FA4E3B1E00E94C92FEAE4F4E756
:104F60000E94CF2F80E080935204A3E5B4E08C919F
:104F70008F5F8C93A1E5B4E08C918F5F8C9300914F
:104F80002A01023118F011F00C94C8270C940B2957
:104F900040912A0100915104041711F00C94D32779
:104FA00081E080935204A0EEB6E0AF93BF93EEE1B0
:104FB000F4E00E9409330E944D3011E001E0BF91FE
:104FC000AF910E948935E0EEF6E0A4E3B1E00E94E3
:104FD0004736EEE1F4E00E940933EAE2F0E70E948E
:104FE0006F340E94783410F00C941128A3E5B4E0DB
:104FF0008C918093620081E080936300A2E5B4E02D
:105000008C9180936400E6E5F5E70E94CF2FA4E33E
:10501000B1E00E94C92FE2E5F4E70E94CF2F0C9483
:105020000329EEE1F4E00E940933EAE2F0E70E948E
:105030006F340E94783481E008F480E08F93EEE1D1
:10504000F4E00E940933EEE6F0E70E946F340E941C
:10505000783481E010F009F080E09F918923882363
:1050600011F40C944E28A3E5B4E08C918093620077
:1050700081E080936300A2E5B4E08C9180936400AA
:10508000E2E6F5E70E94CF2FA4E3B1E00E94C92F2A
:10509000E2E5F4E70E94CF2F0C940329EEE1F4E05F
:1050A0000E940933EEE2F0E70E946F340E947834E8
:1050B00081E008F480E08F93EEE1F4E00E94093390
:1050C000E2E7F0E70E946F340E94783481E010F04C
:1050D00009F080E09F918923882311F40C948B2898
:1050E000A3E5B4E08C918093620081E0809363003B
:1050F000A2E5B4E08C9180936400EEE6F5E70E94AF
:10510000CF2FA4E3B1E00E94C92FE2E5F4E70E94AB
:10511000CF2F0C940329EEE1F4E00E940933E2E37F
:10512000F0E70E946F340E94783481E008F480E058
:105130008F93EEE1F4E00E940933E6E7F0E70E9486
:105140006F340E94783481E010F009F080E09F9184
:105150008923882311F40C94C828A3E5B4E08C912A
:105160008093620081E080936300A2E5B4E08C91BB
:1051700080936400E8E7F5E70E94CF2FA4E3B1E055
:105180000E94C92FE2E5F4E70E94CF2F0C94032977
:10519000EEE1F4E00E940933EAE7F0E70E946F34A1
:1051A0000E94783481E008F480E08F93EEE1F4E02F
:1051B0000E940933EEE7F0E70E946F340E947834D2
:1051C00081E010F009F080E09F918923882311F499
:1051D0000C940329A3E5B4E08C918093620081E0F4
:1051E00080936300A2E5B4E08C9180936400E2E8D0
:1051F000F5E70E94CF2FA4E3B1E00E94C92FE2E5BA
:10520000F4E70E94CF2F80E080935204A3E5B4E03E
:105210008C918F5F8C93A1E5B4E08C918F5F8C9320
:1052200000912A01033118F011F00C9419290C9403
:10523000352940912A0100915104041711F00C9472
:10524000242981E080935204A3E5B4E08C918093FB
:10525000620081E080936300A2E5B4E08C918093CA
:105260006400EAE8F5E70E94CF2F0E940922089522
:1052700000912A010C3011F00C945129ABE2B1E0FD
:105280008C918F5F8C9300912B01063018F011F0F8
:105290000C944C290C944F2986E080932B010C949C
:1052A000622B0D3011F00C94BA29A8ECB0E00D91EE
:1052B0001D912D913C91ABE2B1E0AD90BB24AAE7EA
:1052C000B0E0AA0CBB1CAA0CBB1CAA0DBB1D4D91C7
:1052D0005D916D917C910E94D135A8ECB0E00D9369
:1052E0001D932D933D9342E050E060E070E0A4ED0B
:1052F000B0E00D911D912D913C910E94DB3511F094
:105300000C949829A8ECB0E00D911D912D913C9141
:10531000A4ECB0E04D915D916D917C910E94D135EE
:10532000ACECB0E00D931D932D933D930C94B829F4
:10533000ACECB0E04D915D916D917C91A8ECB0E04A
:105340000D911D912D913C910E94DB351CF011F0C7
:105350000C94AC290C94B829ACECB0E00D911D91E3
:105360002D913C91A8ECB0E00D931D932D933C93AF
:105370000C94622B0E3011F00C94FE29ACECB0E0D2
:105380000D911D912D913C91ABE2B1E0AD90BB240C
:10539000AAE7B0E0AA0CBB1CAA0CBB1CAA0DBB1D43
:1053A0004D915D916D917C910E94D135ACECB0E056
:1053B0000D931D932D933D93ACEBB0E04D915D911A
:1053C0006D917C91ACECB0E00D911D912D913C91D3
:1053D0000E94DB351CF011F00C94F0290C94FC2990
:1053E000ACEBB0E00D911D912D913C91ACECB0E097
:1053F0000D931D932D933C930C94622B0F3011F061
:105400000C94212A41E050E060E070E0A8EDB0E0AB
:105410000D911D912D913C910E94DB3511F00C9462
:10542000192AA8EDB0E0E2E8F0E70E9462350C949A
:105430001F2AA8EDB0E0EAE3F0E70E9462350C9481
:10544000622B003111F00C947A2A41E050E060E0C8
:1054500070E0A4EDB0E00D911D912D913C910E9462
:10546000DB3511F00C94722AA4EDB0E0E2E8F0E72D
:105470000E946235A8ECB0E00D911D912D913C91F8
:10548000A4ECB0E04D915D916D917C910E94D1357D
:10549000ACECB0E00D931D932D933D93ACEBB0E0DD
:1054A0004D915D916D917C91ACECB0E00D911D91B1
:1054B0002D913C910E94DB351CF011F00C94622A76
:1054C0000C946E2AACEBB0E00D911D912D913C91A6
:1054D000ACECB0E00D931D932D933C930E9496315C
:1054E0000C94782AA4EDB0E0EAE3F0E70E9462357C
:1054F0000C94622B013111F00C94E12AA4ECB0E081
:105500000D911D912D913C91ABE2B1E0AD90BB248A
:10551000AAE7B0E0AA0CBB1CAA0CBB1CAA0DBB1DC1
:105520004D915D916D917C910E94D135A4ECB0E0DC
:105530000D931D932D933D9342E050E060E070E0A9
:10554000A4EDB0E00D911D912D913C910E94DB35B1
:1055500011F00C94DF2AA8ECB0E00D911D912D9173
:105560003C91A4ECB0E04D915D916D917C910E94D5
:10557000D135ACECB0E00D931D932D933D93ACEB86
:10558000B0E04D915D916D917C91ACECB0E00D91EE
:105590001D912D913C910E94DB351CF011F00C9473
:1055A000D32A0C94DF2AACEBB0E00D911D912D9124
:1055B0003C91ACECB0E00D931D932D933C930C9477
:1055C000622B023111F00C94F82AA6E2B4E08C911F
:1055D0008F5F8C9300912604053018F011F00C9425
:1055E000F32A0C94F62A85E0809326040C94622B0F
:1055F000033111F00C942E2BE6E2F4E0A190BB24D1
:10560000E2E0F4E0AA0CBB1CAA0CBB1CEA0DFB1DDB
:105610000E940E33EAE1F4E00E9409330E94143440
:10562000FF27EDE0AAE1B4E00E944C36EAE1F4E0A5
:105630000E940933E6E8F0E70E946F340E94783454
:1056400018F011F00C94262B0C942C2BAAE1B4E04A
:10565000E6E8F0E70E9462350C94622B043111F009
:105660000C94622BE6E2F4E0A190BB24E2E0F4E0CB
:10567000AA0CBB1CAA0CBB1CEA0DFB1D0E940E331E
:10568000EEE1F4E00E9409330E941434FF27EDE0BC
:10569000AEE1B4E00E944C36EEE1F4E00E94093342
:1056A000E6E8F0E70E946F340E94783418F011F0B9
:1056B0000C945C2B0C94622BAEE1B4E0E6E8F0E7CE
:1056C0000E946235089500912A010C3011F00C946B
:1056D000792B80912B01815080932B0100912B011C
:1056E000013010F00C94772B81E080932B010C9407
:1056F000C72D0D3011F00C94DE2BA8ECB0E00D910D
:105700001D912D913C91ABE2B1E0AD90BB24AAE795
:10571000B0E0AA0CBB1CAA0CBB1CAA0DBB1D4D9172
:105720005D916D917C910E94D635A8ECB0E00D930F
:105730001D932D933D93A0ECB0E04D915D916D9143
:105740007C91A8ECB0E00D911D912D913C910E94AF
:10575000DB350CF402C00C94B92BA0ECB0E00D9139
:105760001D912D913C91A8ECB0E00D931D932D93CC
:105770003C9342E050E060E070E0A4EDB0E00D91B9
:105780001D912D913C910E94DB3511F00C94DC2B86
:10579000A8ECB0E00D911D912D913C91A4ECB0E0EE
:1057A0004D915D916D917C910E94D135ACECB0E052
:1057B0000D931D932D933D930C94C72D0E3011F036
:1057C0000C94202CACECB0E00D911D912D913C91EE
:1057D000ABE2B1E0AD90BB24AAE7B0E0AA0CBB1CE1
:1057E000AA0CBB1CAA0DBB1D4D915D916D917C91C6
:1057F0000E94D635ACECB0E00D931D932D933D93F4
:10580000A8ECB0E04D915D916D917C91ACECB0E075
:105810000D911D912D913C910E94DB350CF402C03D
:105820000C941E2CA8ECB0E00D911D912D913C9193
:10583000ACECB0E00D931D932D933C930C94C72DCD
:105840000F3011F00C94432C41E050E060E070E028
:10585000A8EDB0E00D911D912D913C910E94DB359A
:1058600011F00C943B2CA8EDB0E0E2E8F0E70E94C8
:1058700062350C94412CA8EDB0E0EAE3F0E70E9419
:1058800062350C94C72D003111F00C949C2C41E032
:1058900050E060E070E0A4EDB0E00D911D912D911D
:1058A0003C910E94DB3511F00C94942CA4EDB0E0F7
:1058B000E2E8F0E70E946235A8ECB0E00D911D919E
:1058C0002D913C91A4ECB0E04D915D916D917C9156
:1058D0000E94D135ACECB0E00D931D932D933D9318
:1058E000ACEBB0E04D915D916D917C91ACECB0E092
:1058F0000D911D912D913C910E94DB351CF011F012
:105900000C94842C0C94902CACEBB0E00D911D9178
:105910002D913C91ACECB0E00D931D932D933C93F5
:105920000E9496310C949A2CA4EDB0E0EAE3F0E7E3
:105930000E9462350C94C72D013111F00C94352D65
:10594000ABE2B1E0AD90BB24AAE7B0E0AA0CBB1C6F
:10595000AA0CBB1CAA0DBB1D4D915D916D917C9154
:10596000A4ECB0E00D911D912D913C910E94DB358E
:105970000CF402C00C94D22CABE2B1E0AD90BB248D
:10598000AAE7B0E0AA0CBB1CAA0CBB1CAA0DBB1D4D
:105990000D911D912D913C91A4ECB0E00D931D93C0
:1059A0002D933C93A4ECB0E00D911D912D913C9171
:1059B000ABE2B1E0AD90BB24AAE7B0E0AA0CBB1CFF
:1059C000AA0CBB1CAA0DBB1D4D915D916D917C91E4
:1059D0000E94D635A4ECB0E00D931D932D933D931A
:1059E00042E050E060E070E0A4EDB0E00D911D9168
:1059F0002D913C910E94DB3511F00C94332DA8ECD5
:105A0000B0E00D911D912D913C91A4ECB0E04D9131
:105A10005D916D917C910E94D135ACECB0E00D931D
:105A20001D932D933D93ACEBB0E04D915D916D9145
:105A30007C91ACECB0E00D911D912D913C910E94B8
:105A4000DB351CF011F00C94272D0C94332DACEBAE
:105A5000B0E00D911D912D913C91ACECB0E00D9317
:105A60001D932D933C930C94C72D023111F00C948F
:105A7000492D8091260481508093260400912604AC
:105A8000013010F00C94472D81E0809326040C9493
:105A9000C72D033111F00C94892DEAE1F4E00E9446
:105AA0000933E6E2F4E0A190BB24E2E0F4E0AA0CC2
:105AB000BB1CAA0CBB1CEA0DFB1D0E940E330E94EE
:105AC000783418F011F00C946D2DE6E0F4E0AAE1C2
:105AD000B4E00E944C360C94872DE6E2F4E0A190ED
:105AE000BB24E2E0F4E0AA0CBB1CAA0CBB1CEA0D30
:105AF000FB1D0E940E33EAE1F4E00E9409330E948C
:105B00000534FF27EDE0AAE1B4E00E944C360C9486
:105B1000C72D043111F00C94C72DEEE1F4E00E9482
:105B20000933E6E2F4E0A190BB24E2E0F4E0AA0C41
:105B3000BB1CAA0CBB1CEA0DFB1D0E940E330E946D
:105B4000783418F011F00C94AD2DEAE0F4E0AEE1F9
:105B5000B4E00E944C360C94C72DE6E2F4E0A1902C
:105B6000BB24E2E0F4E0AA0CBB1CAA0CBB1CEA0DAF
:105B7000FB1D0E940E33EEE1F4E00E9409330E9407
:105B80000534FF27EDE0AEE1B4E00E944C36089505
:105B9000EEEEF3E0D190E0808FEFE7FE8827F82E5D
:105BA000082F0E942D330E946333EAE8F0E70E9439
:105BB00066340E940534FF27EDE0A1EFB3E00E94B8
:105BC0004C36E0EEF3E00E940E33E1EFF3E00E948A
:105BD00009330E94D433FF27EDE0A1EFB3E00E9428
:105BE0004C36A0EEB6E0AF93BF93E1EFF3E00E9436
:105BF00009330E944D3011E001E0BF91AF910E9446
:105C00008935E0EEF6E0A5EFB3E00E944736ACEC54
:105C1000B0E00D911D912D913C91A8ECB0E04D911B
:105C20005D916D917C910E94D635ACE6B0E00D930C
:105C30001D932D933D9341E050E060E070E0A8EDAE
:105C4000B0E00D911D912D913C910E94DB3511F03A
:105C50000C94A52EACE6B0E00D911D912D913C91D8
:105C60004FE750E060E070E00E94E12FACE6B0E06A
:105C70004D935D936D937D93ACE6B0E00D911D91D6
:105C80002D913C91A0E7B0E00D931D932D933C9393
:105C9000ACE6B0E00D911D912D913C91AAEEB3E0E0
:105CA0004D915D9157FB1EF46FEF7FEF02C06627A9
:105CB00077270E948332ACE6B0E00D931D932D93BD
:105CC0003D9300914F01053011F00C948F2EACECF8
:105CD000B0E00D911D912D913C91ACE6B0E04D915D
:105CE0005D916D917C910E94D635ACE6B0E00D934C
:105CF0001D932D933D9305EE13E82EE135E0ACE6C0
:105D0000B0E04D915D916D917C910E94D635ACE6ED
:105D1000B0E00D931D932D933D930C94A32EACE610
:105D2000B0E00D911D912D913C91A8ECB0E04D910A
:105D30005D916D917C910E94D135ACE6B0E00D9300
:105D40001D932D933D930C94342FE8ECF0E00E94CA
:105D500009330E942D33A1EFB3E00E945E33E1EFDF
:105D6000F3E00E940538FF27EDE0A1EFB3E00E94C9
:105D70004C36ECECF0E00E9409330E942D33ABE48A
:105D8000B1E00E945E33EBE4F1E00E940538FF27AA
:105D9000EDE0ABE4B1E00E944C36E1EFF3E00E94AD
:105DA0000E33EBE4F1E00E9409330E940534FF2733
:105DB000EDE0ABE4B1E00E944C36EAE6F0E70E9489
:105DC0006F34EBE4F1E00E9409330E947E33FF2739
:105DD000EDE0ABE4B1E00E944C36EAEEF3E0D190A6
:105DE000E0808FEFE7FE8827F82E082F0E942D33E2
:105DF0000E946333EBE4F1E00E9409330E94D43344
:105E0000FF27EDE0ABE4B1E00E944C36EBE4F1E0BB
:105E10000E940E33E1EFF3E00E9409330E94143434
:105E2000FF27EDE0ABE4B1E00E944C36EBE4F1E09B
:105E30000E940E33EAE2F0E70E9466340E94D037F7
:105E4000FF27EDE0ABE4B1E00E944C36EBE4F1E07B
:105E50000E943037FF27EDE00E94CB32ACE6B0E085
:105E6000EDE0FF270E944C36E2E9F0E00E940933A2
:105E70000E942D330E9463332F933F934F935F9380
:105E8000ECE6F0E00E9409330E942D335F914F91C0
:105E90003F912F910E947E33FF27EDE0ABE4B1E00C
:105EA0000E944C36A0EEB6E0AF93BF93EBE4F1E076
:105EB0000E9409330E944D3011E005E0BF91AF917F
:105EC0000E948935E0EEF6E0A4E3B1E00E94473697
:105ED0008091E8008F7D8093E80008958AE090E04B
:105EE0000E943E300895481A8827580A0895480E9F
:105EF0008827581E0895ED91FC913196FC93EE93FE
:105F00000895ED91FC913197FC93EE93089509D09B
:105F10000E94793200FC10D0089503D01ED001F801
:105F2000F9CF0024E89457FF02C009D0689400F824
:105F30000BD010F80124089502D009D0089550958F
:105F400040954F5F5F4F0895E89417FF08950095BF
:105F500010950F5F1F4F68940895352F242FE894F4
:105F6000452B11F468940895512F402F00271127D5
:105F700080E1440F551F001F111F021B130B4160CE
:105F800018F4020F131F4E7F8A9599F70895A0EE1B
:105F9000B6E08D91882311F00FD0FBCF08950E94B9
:105FA0006234802D11F008D0FACF089588EE93E086
:105FB00065D03197D9F708950C94AA3100FC05D02B
:105FC000089530D005D001F8F9CF37D03FD00895EB
:105FD000842F952FA62FB72FE894452B462B472BC0
:105FE00011F468940895402F512F622F732F0027CA
:105FF000112722273327F0E2440F551F661F771F12
:10600000001F111F221F331F081B190B2A0B3B0BEC
:10601000416028F4080F191F2A1F3B1F4E7FFA9575
:1060200059F708950024E89477FF02C006D06894D9
:1060300000F809D010F80124089512D04F5F5F4F87
:106040006F4F7F4F0895E89437FF0895009510959E
:10605000209530950F5F1F4F2F4F3F4F6894089545
:10606000409550956095709508953197F1F7089592
:10607000689462F80895E89462F80895EF93FF93A6
:10608000EE27E82BE92B31F0E0EDF7E03197F1F75F
:106090000197D1F7FF91EF9108958DE207FD8D9360
:1060A0008F2D881F802F881F8F57082F6894F7F82F
:1060B000802F87FF15C080958395082F80E38D93EF
:1060C0008EE28D93802F815228F080E38D93992763
:1060D0009C93089544270A95802F09F196D01FC0FC
:1060E000805230F09EE49D9381E48D939D93EFCF99
:1060F0004427DF92EF92FF920F938FE1801B11F004
:10610000082F83D089D09EE29D930F91FF90EF904E
:10611000DF9044270395003209F4D7CF2BD03F936B
:10612000EAEAF1E638E12F2D1E2D0D2DFF24EE2495
:10613000DD244427000F111F221FA8F42F923F9245
:106140000E946234102C0E946234202C0E9462341F
:10615000302C0E9462343197410DD21CE31CF01C9C
:106160003F902F9001C0339631963A9519F73F91A1
:1061700007D0AFCFDD0CEE1CFF1C0A95D9F70895B0
:10618000002719E058D08F93802B11F0039501C0A0
:106190008F911A95B9F7802F882309F496CF8F91A4
:1061A000805D8D930A95D9F792CF0065CD1D80B2A1
:1061B000E60E40597307A0ACB90350D6DC01286B3A
:1061C000EE0094357700CA9A3B0065CD1D00B2E61B
:1061D0000E0059730700ACB90300D6DC01006BEE6A
:1061E0000000357700009A3B0000CD1D0000E60E50
:1061F000000073070000B9030000DC010000EE009E
:106200000000770000003B000000F694E794D7946C
:1062100047950A95D1F7089500270DD08F930395E0
:106220008F2D8E298D29842BC1F78F91805D8D93C1
:106230000A95D9F74CCF1F930F93002710E2440F14
:10624000DD1CEE1CFF1C001F802F9AE0890B10F054
:10625000082F43951A9599F7802F0F911F91089554
:10626000442719D0DA98DB9ADD9884E699270E94B2
:106270003E309FEF94BBDA9A30D014FCFDCF02D0B1
:106280004FEF09D08FE310D080EC0ED080E40CD01B
:1062900088EB0AD00895403420F0D89AD998405419
:1062A0000895D99AD8980895DC9801C0DC9AEF93A4
:1062B000FF93E6E0F0E00E943530FF91EF9185BB5F
:1062C000DB98DD9A000000000000000000000000E4
:1062D000000000000000DD980895DC9804D017FC51
:1062E000FCCF0895DC9A992794BB9FEF95BBEF9361
:1062F000FF93E6E0F0E00E943530FF91EF91DB9AEA
:10630000DD9A000000000000000000000000000016
:10631000000000000000000000000000000000007D
:106320000000000013B2DD9894BB08954427B3DF4A
:1063300002D04FEFB0DF00E080E4B6DF88EB800FE3
:10634000B3DF10E48827B2DF1A95E1F70395083030
:1063500099F70895EF93FF93509162005F937090C7
:106360006300E0916000F09161000E946234202D92
:106370000E946234302D0E946234002D319680528A
:10638000482F0E947336E40FF51F70926300732F3D
:1063900040916300509162001DD00E946234802DB4
:1063A00050916400552309F0809580DF509163007F
:1063B0005395509363007A9559F750916200539525
:1063C000509362002A9509F75F9150936200FF9104
:1063D000EF9108954A955A955EDF88EB850F64DF4B
:1063E00080E4840F61CF0F921F922F923F920F9300
:1063F0009F934F93052F48E00E947F36082E4F91C0
:10640000502F242E352EE8DF6DDF6CDF422D532D0B
:10641000E3DF802D0E9472350F91002311F0182ABE
:1064200001C01922812D42DF0F913F902F901F90C4
:106430000F900895AA24BB24FF24EC81EA80EE1A71
:10644000FF08FB81298033242F1A330881E0EA14E6
:10645000FA043CF42FEF3FEFE094F094E80EFA1CBE
:1064600002C021E033272A143A043CF46FEF7FEF97
:1064700020943094280E3A1C02C061E0772735D072
:106480002E143F0414F009F017C0CE2CDF2CCC0CD6
:10649000DD1C022C132C000C111C9A81E91761F0F1
:1064A000E20FA00CB11CAE14BF0424F019F0F60FDB
:1064B000AC18BD081AD0F1CFC22CD32CCC0CDD1CEB
:1064C0000E2C1F2C000C111C9981F91711F4259624
:1064D0000895F60FA00CB11CA214B30424F019F017
:1064E000E20FAC18BD0801D0EFCF4E2F5F2F98817F
:1064F0007ACF0F92B801469F8001479F100D569F9B
:10650000100D0F900895C801D901489F80014A9F3E
:1065100090014B9F202C499F100D211D321D5A9F29
:10652000202C589F100D211D321D599F200D311D0B
:10653000689F200D311D699F300D789F300D0895A3
:106540000E9462340D920020D9F70895369A369948
:10655000FECF369A3699FECF84B195B1089590302A
:1065600041F00D911C91000F111F9A95E1F71C93BA
:106570000E930895903071F00D911D912D913C91E5
:1065800036952795179507959A95D1F73C932E93B5
:106590001E930E9308953DD0992711278F2D880FB4
:1065A00080E8F82A802F881F08F41FEF41F08F57EA
:1065B000082F07FD04C0003240F08FEF01C088278C
:1065C000982FD82EE82EF82E09C08FE1801B082FB7
:1065D000F694E794D79497950A95D1F7112351F043
:1065E0009095D094E094F09481E0980F8827D81E7D
:1065F000E81EF81E0F2DFE2CED2CD92E0895D094F8
:10660000E094F09491E0D90E9927E91EF91E1095B7
:106610000895D190E190F1900191089521913191E7
:10662000419151910895102F90E8FF0C001F092708
:10663000990FF7941078652F90E8440F551F59274C
:10664000990F4795607800380895FF0C90E89027DF
:10665000110F9795F794092F0895102FBD2CDE2C5C
:10666000EF2CF02E11234AF4B094D094E094F094DF
:106670009FEFB91AD90AE90AF90A0EE1FF2039F4A5
:10668000FE2CED2CDB2CBB240850C2F76BC032F083
:106690000A95BB0CDD1CEE1CFF1CF9CF01D0D5CF39
:1066A000B7FE089590E8B91611F4D0FE08959FEF53
:1066B000D91AE90AF90A09F403950895DD92ED92D1
:1066C000FD920C930895502F2D2D3E2D4F2D612FAF
:1066D00008952DEC3CEC4CEC5DE366270FC099DF90
:1066E000F2DFDD24EE2490E8F92E0FE307C096DFF9
:1066F00005C02227332740E251E46627552351F194
:10670000002381F190DF71F116270058505808944A
:10671000050B18F407FD03C025C007FD23C04695EF
:1067200037952795F694E794D79422D0FF202AF046
:10673000DD0CEE1CFF1C015073F09D2D969548F06A
:10674000DD203AF4EE202AF491E0D90E9927E91ED3
:10675000F91E7BCF07C09FE7092FF92A9FEFD92E9B
:10676000E92E0895DD24EE24FF2400271127089543
:106770009F929924AA24BB2488E1D216E306F4064A
:1067800028F0D21AE30AF40A089401C08894991CEC
:10679000AA1CBB1CDD0CEE1CFF1C8A9571F7D92CC2
:1067A000EA2CFB2C9F9008953EDFE1F25038D1F2A5
:1067B0001627005850580894051F12F418F4CBCF30
:1067C00008F0D0CF0AD0FF202AF0BB0CDD1CEE1C55
:1067D000FF1C3BCF0F5FFBF138CF9F929924AA2477
:1067E000BB24992788E1990CAA1CBB1CDD1CEE1C5C
:1067F000FF1C30F4920EA31EB41ED91EE91EF91E12
:106800008A9589F79F90089509DF0DDF503829F0A8
:1068100090E869270CC00AF045D017CF5FE3222724
:106820003327442701C0FADEFEDE5038B1F30038CA
:1068300099F3902F951B8BF312F434D0FACF983143
:1068400018F0222733274427983028F0232F342F9D
:1068500044279850F9CF992329F0469537952795E5
:106860009A95D9F7912F962742F014D0B0F6F79465
:10687000E794D7940F5F8BF66ECF10D051F008F4E9
:10688000BEDEFF2052F2DD0CEE1CFF1C0150CBF7E8
:1068900062CF68CFD20EE31EF41E0895D21AE30A27
:1068A000F40A0895DF92EF92FF920F931F93D22E76
:1068B000E32EF42E052F162F6F915F914F913F918C
:1068C0002F910895C895319600200895FBDFD02CB4
:1068D000F9DFE02CF7DFF02CF5DF002D0895F2DF73
:1068E000202DF0DF302DEEDF402DECDF502D089510
:1068F00007FB00680EF40F7757FB50680EF45F77C4
:1069000007FD02C057FF05C0D216E306F4060507CF
:1069100008952D153E054F05500708950E943B3000
:10692000E89488278A938A931DDF11278D918032FE
:10693000E9F31197BBD098F08D3229F41095119698
:106940008C91B4D060F08E3229F411968C91AED037
:1069500008F446C022960E94383081E008958C9158
:10696000A5D0D8F547D01196D0F703958D919ED03C
:10697000E0F38E3229F48C9199D010F41196FBCF6C
:10698000853419F0853609F055C011968C918ED05A
:1069900060F08D3219F08B3221F0DCCF088000944A
:1069A000088211968C9182D0A8F680538983119623
:1069B0008C917CD058F49981990F990F0980900D92
:1069C000990F8053890F8983873220F689819881B6
:1069D00099230AF48195080F2DC08E3289F61196FD
:1069E0008C9164D068F606D018F011960A95F8CF0D
:1069F0001196C1CF4F2D3E2D2D2DDD0CEE1CFF1C11
:106A0000A8F0DD0CEE1CFF1C88F0D20EE31EF41E75
:106A100068F0DD0CEE1CFF1C48F0805309F0689410
:106A2000D80E8827E81EF81E08F00895F42EE32EED
:106A3000D22E089534D019F116F5098308E921D032
:106A40000695882787959F2D9F77980FF92E0150DF
:106A5000000F110F07958981882379F01AF4819529
:106A6000898306C036DE89818A958983D9F705C076
:106A700040DE89818A958983D9F72296089572DE4E
:106A8000FCCF0DD041F0FF2032F00A9531F0DD0C43
:106A9000EE1CFF1CD2F788940895089408950024F2
:106AA0000D280E280F28002A00200895803320F09A
:106AB0008A3310F4089408958894089591E005C0ED
:106AC00092E003C094E001C098E0FCDE0D929A953C
:106AD000E1F7089582E001C084E099279D938A95AB
:106AE000E9F7089591E0882321F08894991F8A9509
:106AF000E9F7892F9095089599278D91939588238B
:106B0000E1F7939511968C9311978E919A95D1F701
:106B10000895EA2FFB2F00244C918D9103948E321F
:106B2000E1F711248D9113948823E1F71A9410163C
:106B300040F41197202F2119239580E38D932A95F6
:106B4000E9F7113039F59927AE2FBF2FA00DB91FE6
:106B5000A00FB91F8C919C93853308F421C031E0BC
:106B60008E918E32E9F38D3241F0830F8A3319F41E
:106B700080E331E001C033278C93AE1789F73323CC
:106B800041F0AE2FBF2FB8DF81E34D3209F43196CB
:106B9000808308958827E00DF81FE00FF81F808399
:106BA0000895040F151F261F371F0895041B150B8A
:106BB000260B370B08950417150726073707089586
:106BC000000F111F221F331F089500951095209567
:106BD00030950F5F1F4F2F4F3F4F08950191108148
:106BE0000EC001911191219130810BC00191108152
:106BF00017FF05C03FEF2FEF04C0008111272227A8
:106C0000332737FF03C0E1DF8DE28D93CF93DF930E
:106C1000CF92DF92EF92AA24BB24CC24DD24EE2471
:106C200040E2CAE0DD2755E093E38881890F87FDC4
:106C30009F7083FD907F891B89935A95A9F7C0DFC8
:106C4000AA1CBB1CCC1CDD1CEE1C4A9551F7E89419
:106C5000EFE0FF2782910ED0EB30E0F71EF0689452
:106C60008A2D0CD088278D93EF90DF90CF90DF9105
:106C7000CF910895982F829501D0892F8F70805DD4
:106C800026F0803309F4089568948D9308958191D6
:106C90008D938823E1F7089594E081918D939A95DF
:106CA000E1F70895E199FECFEEBBFFBB3196089561
:106CB00091E001C092E07B3751F47FB7F894F2DFA6
:106CC0008D918DBBE29AE19A9A95C9F77FBF77279C
:106CD000089591E001C092E0E5DFE09A8DB38D93D5
:106CE0009A95D1F70895FF935527F8E0469508F453
:106CF000500F57954795FA95D1F7FF910895FF9357
:106D0000881BF9E0001FFA9511F4FF910895881F80
:106D1000841B18F4840F8894F5CF0894F3CF0027D0
:106D200011272D913D910217130714F4022F132FF1
:106D30003197B9F708950FEF1FEF2D913D9102178D
:106D4000130710F0022F132F3197B9F708950FEFA3
:106D50001FEF88279927442755272D913D910196AC
:106D60000217130720F0022F132F482F592F3197A6
:106D7000A1F708954EDC57DC0395AAF087E1DD0CFE
:106D8000EE1CFF1C8A9589F00A95CAF7FF205AF07D
:106D900000240D280E280F28002039F00A95DD0C5C
:106DA000EE1CFF1CDAF70A9550CCDCCCDBCC31DCD6
:106DB0000023E2F374DE19F4CEDC0068089585E068
:106DC00011D1FF0C001F04830FE70695F79424D11F
:106DD00050682ADD73DC139721E438E743ED5BEB61
:106DE000E3DC27E831ED43E15DE3D6D02EE03CE380
:106DF00043EC5DEBD1D022E83DEA4BE25EE3CCD040
:106E00002CEE32E846E75EEBC7D020E931EE49EAE6
:106E10005EE3C2D020E83FEE4FEF5EEBBDD024EC46
:106E20003FEF4FE75FE3B8D049DC139784818F577A
:106E300099F02AF4D82E0FEFE02EF02E04C0D82EB1
:106E4000EE24FF24002709DC28E132E741E35FE379
:106E5000ABDCE4DB3497E8DCD2C0DBDB80E003C0F2
:106E6000D8DB802F8078882321F0DF92EF92FF9289
:106E70000F938F93D8DB802F839512F473DC1BC0A4
:106E800080958A95885E0AF415C088501AF40CD053
:106E9000D92210C0DD2488501AF406D0E9220AC095
:106EA000EE2402D0F92206C09FEF8770990F8A95D1
:106EB000EAF70895CADB8F918823D9F35F914F9148
:106EC0003F912F910F9314DD0F9199F390F3A4D07C
:106ED0005068AACC40DC93C09CDB86E083D005835D
:106EE0000F772BE33AEA48EB5FE35EDCE7DB1397CF
:106EF00041D028F4858188236AF734DC80C08F77FD
:106F0000848387DB349737DFD9DB139723E632E4BA
:106F100046E357EB49DC29ED37EA4AE159E33CD037
:106F200026E538E14EEA5AEB37D026E53CE84DE15C
:106F30005CE332D02DEC37E543E65DEB2DD02DEE52
:106F40003DEF45E75EE328D028E132E741E35FEB20
:106F500023D062D069DCB7DBDD24EE24FF2404817A
:106F60008FE7080F0695F794C9DB8581881F08F421
:106F7000B7DB45C058DB8827039512F48894089541
:106F800007301AF0812F08940895FF1C881F0A9576
:106F9000E2F7812B8894089547DC40DB349704CCDA
:106FA0007EDD81F00F930F772F933F934F935F9385
:106FB000FFDE5F914F913F912F91F6DB8EDF8F9136
:106FC0008078082B089525DB0F93AF93BF930F773D
:106FD000EFDEFF91EF9122DBE7DB7FDF8F9180789F
:106FE000082B08950FB6F8944A925A92E42DF52D85
:106FF000A42DB52D480E8827581E0FBE08950FB634
:10700000F894599049900FBE089503DBD1DE29ED25
:107010003BE54EED5EE3C8CB5FE340E83327222734
:107020000895CDCCCC3D0000803F00002041000001
:10703000C84200007A440AD7234A01000000000039
:10704000A04082E2473E0000004400005C42000095
:107050006442000000BF000080BF0000A0417AE54C
:107060001D42BD378635002474490000FE42CDCC58
:10707000C7429AF979449A3F1C4600401C46F34F98
:10708000C34702000000804FC3470000E0402031AA
:1070900030487A00313030487A0020316B487A002D
:1070A00031306B487A00203130306B0020314D4850
:1070B0007A0020202020204E412D30312020202019
:1070C000202000006369726375697420616E616CD1
:1070D000797A657200002020207665722E20352E88
:1070E0003535202020200000206D61646520627904
:1070F000207370366672652000002D2D2D2D2D2DEC
:107100002D2D2D2D2D2D2D2D2D2D000068747470FD
:107110003A2F2F6C782D6E65742E706C00004F4BDB
:107120000000506F6D6961722077207061736D6926
:107130006500506F6D696172202B20510000506F07
:107140006D696172206D6F6379004D6F7374656B4B
:107150002053575200004D6F6E69746F72004B617F
:107160006C69627261636A6100004B616C69627292
:1071700061636A6120535752000057796A736369EB
:10718000650057796B6F6E616A206B6F6C656A6E14
:107190006F3A0000312E4F646C61637A2077656A24
:1071A000736369650000322E4E616369736E696AAC
:1071B00020454E5445520000437A792077796B6F11
:1071C0006E6163006B616C69627261636A65206DF8
:1071D0006F63793F0000506F6D696172202020203D
:1071E00020202020202000004B616C6962726163C6
:1071F0006A612020202020200000312E4F646C6125
:10720000637A206F64205765202000007A726F64D3
:107210006C6F206D6F637920202020200000312EBC
:10722000446F6C61637A20646F20576520200000F2
:1072300020207A726F646C6F206D6F63792020203C
:107240000000322E557A796A203C2D2020692020BA
:107250002D3E0000202069207573746177206D6FCA
:1072600063206D570000332E205A616B6F6E637A76
:1072700020454E54455200004D6F632077206D57D6
:10728000203D200020202020202020202020202001
:10729000202020200000202020202020202020202E
:1072A000000075572000572000006D5720006442F1
:1072B0006D00557A796A206D6F73746B6120535736
:1072C000523A0000312E506F6C61637A205779205A
:1072D0004E413032000020207A205765206D6F73B8
:1072E000746B612020200000322E506F6C61637A35
:1072F000205765204E413032000020207A204D6F0B
:107300006E206D6F73746B6120200000332E446F0C
:107310006C61637A20646F20577920200000202060
:107320006D6F73746B61203530206F686D200000C5
:10733000342E4E616369736E696A20454E5445521E
:107340000000557A796A2070727A79737461776B6C
:10735000693A0000312E5573756E207A20676E6988
:10736000617A642000002020656C656D656E74791B
:107370002020202020200000312E506F6C61637A85
:10738000207765207A2077790000557A796A206D18
:107390006F73746B61205357523A2000312E4F6443
:1073A0006C61637A206F64205779202000004B6F56
:1073B0006E696563206B616C6962722E0000777381
:1073C00074617720646F20676E69617A640062611E
:1073D00064616E6520656C656D656E747900446FDF
:1073E0006C61637A20646F20577900006261646188
:1073F0006E7920756B6C616400004D494E203D2014
:1074000000004D4158203D20000044796E203D2071
:107410000000206442004D20000064420000494EFC
:107420004600202020202020205357523D004D6947
:107430006E3D0000496E643D000046723D004D48BF
:107440007A00513D00004C783D00754800004378BB
:107450003D00704600004D00506F6D696172200064
:10746000537465703A2020202020200053746172EC
:107470003A202000537461723A20000053746F70F8
:107480003A20200053746F703A2000004C494E009F
:107490004C4F4700537761703A2020202020202055
:1074A0002000532F530044454C004D6F64653A2033
:1074B000202020202020200044656C743A202000E9
:1074C00044656C743A2000004C4373743A202020C9
:1074D0002020202020302E3100004C4373743A20AD
:1074E0002020202020202020203100004C437374D5
:1074F0003A202020202020202020313000004C4342
:1075000073743A20202020202020203130300000C9
:107510004C4373743A20202020202020313030301A
:1075200000004C7220203A202020202020004C72A5
:1075300020203A202020202000004C7220203A20D9
:10754000202020004C7220203A20202000004C7285
:1075500020203A202000437220203A2020202020A2
:107560002000437220203A20202020200000437277
:1075700020203A2020202000437220203A20202082
:107580000000437220203A2020005341564520201D
:047590002020200097
:00000001FF
